 hcd_hsh2

 Timestamp is 4da293b5 (Mon Apr 11 17:37:57 2011)

 Preferred load address is 10000000

 Start         Length     Name                   Class
 0001:00000000 00000004H .CRT$XCA                CODE
 0001:00000004 00000004H .CRT$XCZ                CODE
 0001:00000008 00000004H .CRT$XIA                CODE
 0001:0000000c 00000004H .CRT$XIZ                CODE
 0001:00000010 00000004H .CRT$XPA                CODE
 0001:00000014 00000004H .CRT$XPZ                CODE
 0001:00000018 00000004H .CRT$XTA                CODE
 0001:0000001c 00000004H .CRT$XTZ                CODE
 0001:00000020 000008e2H .rdata                  CODE
 0001:00000904 00000025H .rdata$debug            CODE
 0001:0000092c 00010708H .text                   CODE
 0001:00011034 00000184H .xdata                  CODE
 0001:000111b8 0000003cH .idata$2                CODE
 0001:000111f4 00000014H .idata$3                CODE
 0001:00011208 00000140H .idata$4                CODE
 0001:00011348 000000d4H .idata$6                CODE
 0001:00011420 00000100H .edata                  CODE
 0002:00000000 00000140H .idata$5                DATA
 0002:00000140 00000114H .data                   DATA
 0002:00000260 00000090H .bss                    DATA
 0003:00000000 00000d80H .pdata                  DATA

  Address         Publics by Value              Rva+Base       Lib:Object

 0000:00000000       ___safe_se_handler_count   00000000     <absolute>
 0000:00000000       ___safe_se_handler_table   00000000     <absolute>
 0001:00000000       __xc_a                     10001000     corelib0:crt0init.obj
 0001:00000004       __xc_z                     10001004     corelib0:crt0init.obj
 0001:00000008       __xi_a                     10001008     corelib0:crt0init.obj
 0001:0000000c       __xi_z                     1000100c     corelib0:crt0init.obj
 0001:00000010       __xp_a                     10001010     corelib0:crt0init.obj
 0001:00000014       __xp_z                     10001014     corelib0:crt0init.obj
 0001:00000018       __xt_a                     10001018     corelib0:crt0init.obj
 0001:0000001c       __xt_z                     1000101c     corelib0:crt0init.obj
 0001:0000003c       ??_C@_1CC@BJPGGDNC@?$AAU?$AAS?$AAB?$AA_?$AAC?$AAL?$AAO?$AAC?$AAK?$AA_?$AAG?$AAA?$AAT?$AAI?$AAN?$AAG?$AA?$AA@ 1000103c     i_usbclock.obj
 0001:00000060       ??_C@_1BI@BHLBGEOK@?$AAP?$AAr?$AAi?$AAo?$AAr?$AAi?$AAt?$AAy?$AA2?$AA5?$AA6?$AA?$AA@ 10001060     usbh_usb2com_common_topaz_v1:hcddrv.obj
 0001:00000078       ??_C@_17KACEIPNC@?$AAK?$AAe?$AAy?$AA?$AA@ 10001078     usbh_usb2com_common_topaz_v1:hcddrv.obj
 0001:00000080       ??_7CHcd@@6B@              10001080     usbh_usb2com_common_topaz_v1:hcd.obj
 0001:000000f0       ??_C@_1CA@GOGEMIHH@?$AAW?$AAa?$AAi?$AAt?$AAF?$AAo?$AAr?$AAA?$AAP?$AAI?$AAR?$AAe?$AAa?$AAd?$AAy?$AA?$AA@ 100010f0     usbh_usb2com_common_topaz_v1:cdevice.obj
 0001:00000110       ??_C@_1BM@LLINKHBA@?$AAk?$AA?4?$AAc?$AAo?$AAr?$AAe?$AAd?$AAl?$AAl?$AA?4?$AAd?$AAl?$AAl?$AA?$AA@ 10001110     usbh_usb2com_common_topaz_v1:cdevice.obj
 0001:0000012c       ??_C@_1BO@KLPJMMP@?$AAC?$AAe?$AAC?$AAa?$AAl?$AAl?$AAU?$AAs?$AAe?$AAr?$AAP?$AAr?$AAo?$AAc?$AA?$AA@ 1000112c     usbh_usb2com_common_topaz_v1:cdevice.obj
 0001:0000014c       ??_7CDeviceGlobal@@6B@     1000114c     usbh_usb2com_common_topaz_v1:cdevice.obj
 0001:0000015c       ??_C@_1BE@NANPENDH@?$AAH?$AAc?$AAd?$AAA?$AAt?$AAt?$AAa?$AAc?$AAh?$AA?$AA@ 1000115c     usbh_usb2com_common_topaz_v1:cdevice.obj
 0001:00000170       ??_C@_1CE@MBINLHH@?$AAH?$AAc?$AAd?$AAD?$AAe?$AAv?$AAi?$AAc?$AAe?$AAA?$AAt?$AAt?$AAa?$AAc?$AAh?$AAe?$AAd?$AA?$AA@ 10001170     usbh_usb2com_common_topaz_v1:cdevice.obj
 0001:00000194       ??_C@_1CE@KAKNBFJP@?$AAH?$AAc?$AAd?$AAD?$AAe?$AAv?$AAi?$AAc?$AAe?$AAD?$AAe?$AAt?$AAa?$AAc?$AAh?$AAe?$AAd?$AA?$AA@ 10001194     usbh_usb2com_common_topaz_v1:cdevice.obj
 0001:000001b8       ??_C@_1CO@MCCAIHAO@?$AAH?$AAc?$AAd?$AAS?$AAe?$AAl?$AAe?$AAc?$AAt?$AAC?$AAo?$AAn?$AAf?$AAi?$AAg?$AAu?$AAr?$AAa?$AAt?$AAi?$AAo?$AAn?$AA?$AA@ 100011b8     usbh_usb2com_common_topaz_v1:cdevice.obj
 0001:000001e8       ??_C@_1BC@MPAIGMIO@?$AAU?$AAS?$AAB?$AAD?$AA?4?$AAD?$AAL?$AAL?$AA?$AA@ 100011e8     usbh_usb2com_common_topaz_v1:cdevice.obj
 0001:000001fc       ??_C@_1BE@MDMBICMJ@?$AAH?$AAc?$AAd?$AAD?$AAe?$AAt?$AAa?$AAc?$AAh?$AA?$AA@ 100011fc     usbh_usb2com_common_topaz_v1:cdevice.obj
 0001:00000210       ??_7CDevice@@6B@           10001210     usbh_usb2com_common_topaz_v1:cdevice.obj
 0001:00000248       ??_C@_1BK@GALBKKNF@?$AAN?$AAe?$AAt?$AAM?$AAs?$AAg?$AAB?$AAo?$AAx?$AAE?$AAx?$AAt?$AA?$AA@ 10001248     usbh_usb2com_common_topaz_v1:cdevice.obj
 0001:00000264       ??_C@_1BE@BOHEBICI@?$AAn?$AAe?$AAt?$AAu?$AAi?$AA?4?$AAd?$AAl?$AAl?$AA?$AA@ 10001264     usbh_usb2com_common_topaz_v1:cdevice.obj
 0001:00000278       ??_C@_1BE@KCBNNJPA@?$AAU?$AAS?$AAB?$AAD?$AAe?$AAt?$AAa?$AAc?$AAh?$AA?$AA@ 10001278     usbh_usb2com_common_topaz_v1:cdevice.obj
 0001:00000290       ??_7CHub@@6B@              10001290     usbh_usb2com_common_topaz_v1:cdevice.obj
 0001:000002f0       ??_7CRootHub@@6B@          100012f0     usbh_usb2com_common_topaz_v1:cdevice.obj
 0001:00000350       ??_7CExternalHub@@6B@      10001350     usbh_usb2com_common_topaz_v1:cdevice.obj
 0001:000003b0       ??_7CFunction@@6B@         100013b0     usbh_usb2com_common_topaz_v1:cdevice.obj
 0001:000003e8       ??_C@_1HE@EAEFIBJD@?$AAE?$AAx?$AAc?$AAe?$AAe?$AAd?$AA?5?$AAp?$AAo?$AAw?$AAe?$AAr?$AA?5?$AAl?$AAi?$AAm?$AAi?$AAt?$AAa?$AAt?$AAi?$AAo?$AAn?$AA?0?$AA?5?$AAU?$AAS?$AAB?$AA?5?$AAd?$AAe?$AAv@ 100013e8     usbh_usb2com_common_topaz_v1:cdevice.obj
 0001:00000460       ??_C@_1GK@IHAKGPKC@?$AAT?$AAo?$AAo?$AA?5?$AAm?$AAa?$AAn?$AAy?$AA?5?$AAh?$AAu?$AAb?$AA?5?$AAt?$AAi?$AAe?$AAr?$AAs?$AA?0?$AA?5?$AAU?$AAS?$AAB?$AA?5?$AAd?$AAe?$AAv?$AAi?$AAc?$AAe?$AA?5?$AAc@ 10001460     usbh_usb2com_common_topaz_v1:cdevice.obj
 0001:000004d0       ??_7CEhcd@@6B@             100014d0     usbh_ehcdmdd_common_topaz_v1:cehcd.obj
 0001:00000548       ??_7CQTransfer@@6B@        10001548     usbh_ehcdmdd_common_topaz_v1:cpipe.obj
 0001:00000554       ??_7CPipeAbs@@6B@          10001554     usbh_ehcdmdd_common_topaz_v1:cpipe.obj
 0001:00000578       ??_7CPipe@@6B@             10001578     usbh_ehcdmdd_common_topaz_v1:cpipe.obj
 0001:000005b0       ??_7CQueuedPipe@@6B@       100015b0     usbh_ehcdmdd_common_topaz_v1:cpipe.obj
 0001:000005f0       ??_7CBulkPipe@@6B@         100015f0     usbh_ehcdmdd_common_topaz_v1:cpipe.obj
 0001:00000630       ??_C@_19PBJLGAMD@?$AAB?$AAu?$AAl?$AAk?$AA?$AA@ 10001630     usbh_ehcdmdd_common_topaz_v1:cpipe.obj
 0001:00000640       ??_7CControlPipe@@6B@      10001640     usbh_ehcdmdd_common_topaz_v1:cpipe.obj
 0001:00000680       ??_C@_1BA@JGFNDEFA@?$AAC?$AAo?$AAn?$AAt?$AAr?$AAo?$AAl?$AA?$AA@ 10001680     usbh_ehcdmdd_common_topaz_v1:cpipe.obj
 0001:00000690       ??_7CInterruptPipe@@6B@    10001690     usbh_ehcdmdd_common_topaz_v1:cpipe.obj
 0001:000006d0       ??_C@_1BE@PBKDACKD@?$AAI?$AAn?$AAt?$AAe?$AAr?$AAr?$AAu?$AAp?$AAt?$AA?$AA@ 100016d0     usbh_ehcdmdd_common_topaz_v1:cpipe.obj
 0001:000006e4       ??_7CIsochronousPipe@@6B@  100016e4     usbh_ehcdmdd_common_topaz_v1:cpipe.obj
 0001:0000071c       ??_C@_1BI@FKFHNGHF@?$AAI?$AAs?$AAo?$AAc?$AAh?$AAr?$AAo?$AAn?$AAo?$AAu?$AAs?$AA?$AA@ 1000171c     usbh_ehcdmdd_common_topaz_v1:cpipe.obj
 0001:0000073c       ??_7CDummyPipe@@6B@        1000173c     usbh_ehcdmdd_common_topaz_v1:chw.obj
 0001:00000774       ??_C@_1M@EOJMLNDL@?$AAD?$AAu?$AAm?$AAm?$AAy?$AA?$AA@ 10001774     usbh_ehcdmdd_common_topaz_v1:chw.obj
 0001:00000780       ??_C@_1BM@CBMLCADC@?$AAI?$AAn?$AAt?$AAT?$AAh?$AAr?$AAe?$AAs?$AAh?$AAC?$AAt?$AAr?$AAl?$AA?$AA@ 10001780     usbh_ehcdmdd_common_topaz_v1:chw.obj
 0001:000007a0       ??_7CHW@@6B@               100017a0     usbh_ehcdmdd_common_topaz_v1:chw.obj
 0001:00000818       ??_C@_1BA@MLDLNLBG@?$AAU?$AAS?$AAB?$AAH?$AAo?$AAs?$AAt?$AA?$AA@ 10001818     usbh_ehcdmdd_common_topaz_v1:chw.obj
 0001:00000828       ??_C@_1BA@JAHEEJIA@?$AAU?$AAS?$AAB?$AAX?$AAC?$AAV?$AAR?$AA?$AA@ 10001828     usbh_ehcdmdd_common_topaz_v1:chw.obj
 0001:00000838       ??_7CTransfer@@6B@         10001838     usbh_ehcdmdd_common_topaz_v1:trans.obj
 0001:00000844       ??_7CIsochTransfer@@6B@    10001844     usbh_ehcdmdd_common_topaz_v1:trans.obj
 0001:00000860       ??_7CITransfer@@6B@        10001860     usbh_ehcdmdd_common_topaz_v1:trans.obj
 0001:0000087c       ??_7CSITransfer@@6B@       1000187c     usbh_ehcdmdd_common_topaz_v1:trans.obj
 0001:00000898       ??_C@_1CC@NPEFILDH@?$AAP?$AAh?$AAy?$AAs?$AAi?$AAc?$AAa?$AAl?$AAP?$AAa?$AAg?$AAe?$AAS?$AAi?$AAz?$AAe?$AA?$AA@ 10001898     usbh_ehcdpdd_common_topaz_v1:system.obj
 0001:000008bc       ??_C@_1BM@KKKMKIHE@?$AAH?$AAc?$AAd?$AAC?$AAa?$AAp?$AAa?$AAb?$AAi?$AAl?$AAi?$AAt?$AAy?$AA?$AA@ 100018bc     usbh_ehcdpdd_common_topaz_v1:system.obj
 0001:000008d8       ??_C@_1BC@GDFGLIEL@?$AAO?$AAT?$AAG?$AAG?$AAr?$AAo?$AAu?$AAp?$AA?$AA@ 100018d8     usbh_ehcdpdd_common_topaz_v1:system.obj
 0001:000008ec       ??_C@_1BG@HHFAGDDC@?$AAO?$AAT?$AAG?$AAS?$AAu?$AAp?$AAp?$AAo?$AAr?$AAt?$AA?$AA@ 100018ec     usbh_ehcdpdd_common_topaz_v1:system.obj
 0001:0000092c       SetPHYPowerMgmt            1000192c f   i_hwinit.obj
 0001:00000b14       gfnGetOTGGroup             10001b14 f   i_hwinit.obj
 0001:00000b20       gfnIsOTGSupport            10001b20 f   i_hwinit.obj
 0001:00000b30       InitializeTransceiver      10001b30 f   i_hwinit.obj
 0001:00000c58       BSPUsbhCheckConfigPower    10001c58 f   i_hwinit.obj
 0001:00000c6c       BSPUsbCheckWakeUp          10001c6c f   i_hwinit.obj
 0001:00000d10       BSPUsbHostLowPowerModeEnable 10001d10 f   i_hwinit.obj
 0001:00000d18       BSPUSBHostVbusControl      10001d18 f   i_hwinit.obj
 0001:00000da4       BSPNeedCloseVBus           10001da4 f   i_hwinit.obj
 0001:00000dac       IsLowPowerSameAsSuspend    10001dac f   i_hwinit.obj
 0001:00000db4       BSPGetUSBControllerType    10001db4 f   i_hwinit.obj
 0001:00000dbc       BSPUsbSetWakeUp            10001dbc f   i_hwinit.obj
 0001:00000edc       USBClockGatingLock         10001edc f   i_usbclock.obj
 0001:00000f18       BSPUSBClockCreateFileMapping 10001f18 f   i_usbclock.obj
 0001:00000fb8       BSPUSBClockSwitch          10001fb8 f   i_usbclock.obj
 0001:000010ac       USBClockInit               100020ac f   i_usbclock.obj
 0001:000010b4       PowerDownSchemeExist       100020b4 f   i_usbutils.obj
 0001:00001110       BSPUsbEnableLowPowerIntr   10002110 f   i_usbutils.obj
 0001:00001164       BSPUsbSetBusConfig         10002164 f   i_usbutils.obj
 0001:00001174       BSPUSBInterruptControl     10002174 f   i_usbutils.obj
 0001:000011b8       BSPHostDisconDetect        100021b8 f   i_usbutils.obj
 0001:000011bc       DllMain                    100021bc f   usbh_usb2com_common_topaz_v1:hcddrv.obj
 0001:00001214       HcdGetFrameNumber          10002214 f   usbh_usb2com_common_topaz_v1:hcddrv.obj
 0001:00001228       HcdGetFrameLength          10002228 f   usbh_usb2com_common_topaz_v1:hcddrv.obj
 0001:0000123c       HcdSetFrameLength          1000223c f   usbh_usb2com_common_topaz_v1:hcddrv.obj
 0001:00001250       HcdStopAdjustingFrame      10002250 f   usbh_usb2com_common_topaz_v1:hcddrv.obj
 0001:00001264       HcdOpenPipe                10002264 f   usbh_usb2com_common_topaz_v1:hcddrv.obj
 0001:00001268       HcdClosePipe               10002268 f   usbh_usb2com_common_topaz_v1:hcddrv.obj
 0001:0000126c       HcdResetPipe               1000226c f   usbh_usb2com_common_topaz_v1:hcddrv.obj
 0001:00001270       HcdIsPipeHalted            10002270 f   usbh_usb2com_common_topaz_v1:hcddrv.obj
 0001:00001274       HcdIssueTransfer           10002274 f   usbh_usb2com_common_topaz_v1:hcddrv.obj
 0001:00001320       HcdAbortTransfer           10002320 f   usbh_usb2com_common_topaz_v1:hcddrv.obj
 0001:0000136c       HcdMdd_CreateHcdObject_Customized 1000236c f   usbh_usb2com_common_topaz_v1:hcddrv.obj
 0001:000013cc       HcdMdd_DestroyHcdObject    100023cc f   usbh_usb2com_common_topaz_v1:hcddrv.obj
 0001:000013ec       HcdMdd_DestroyMemoryObject 100023ec f   usbh_usb2com_common_topaz_v1:hcddrv.obj
 0001:00001410       HcdMdd_PowerUp             10002410 f   usbh_usb2com_common_topaz_v1:hcddrv.obj
 0001:0000142c       HcdMdd_PowerDown           1000242c f   usbh_usb2com_common_topaz_v1:hcddrv.obj
 0001:00001448       HcdMdd_SetCapability       10002448 f   usbh_usb2com_common_topaz_v1:hcddrv.obj
 0001:0000145c       HcdMdd_SetSubHubTestMode   1000245c f   usbh_usb2com_common_topaz_v1:hcddrv.obj
 0001:000014a4       HCD_Init                   100024a4 f   usbh_usb2com_common_topaz_v1:hcddrv.obj
 0001:000015e4       HCD_PowerUp                100025e4 f   usbh_usb2com_common_topaz_v1:hcddrv.obj
 0001:000015e8       HCD_PowerDown              100025e8 f   usbh_usb2com_common_topaz_v1:hcddrv.obj
 0001:000015ec       HCD_Deinit                 100025ec f   usbh_usb2com_common_topaz_v1:hcddrv.obj
 0001:000015f0       HCD_Open                   100025f0 f   usbh_usb2com_common_topaz_v1:hcddrv.obj
 0001:000015f4       HCD_Close                  100025f4 f   usbh_usb2com_common_topaz_v1:hcddrv.obj
 0001:000015f8       HCD_Read                   100025f8 f   usbh_usb2com_common_topaz_v1:hcddrv.obj
 0001:000015fc       HCD_Write                  100025fc f   usbh_usb2com_common_topaz_v1:hcddrv.obj
 0001:00001600       HCD_Seek                   10002600 f   usbh_usb2com_common_topaz_v1:hcddrv.obj
 0001:00001604       HCD_IOControl              10002604 f   usbh_usb2com_common_topaz_v1:hcddrv.obj
 0001:00001630       HcdMdd_CreateMemoryObject  10002630 f   usbh_usb2com_common_topaz_v1:hcddrv.obj
 0001:000016ac       ??0CHcd@@QAA@XZ            100026ac f   usbh_usb2com_common_topaz_v1:hcd.obj
 0001:000016e0       ?WaitForPortStatusChange@CHcd@@UAAHPAX@Z 100026e0 f i usbh_usb2com_common_topaz_v1:hcd.obj
 0001:000016e8       ?SuspendHC@CHcd@@UAAHXZ    100026e8 f i usbh_usb2com_common_topaz_v1:hcd.obj
 0001:000016f0       ?ResumeNotification@CHcd@@MAAHXZ 100026f0 f i usbh_usb2com_common_topaz_v1:hcd.obj
 0001:00001738       ??1CHcd@@UAA@XZ            10002738 f   usbh_usb2com_common_topaz_v1:hcd.obj
 0001:000017ac       ?SetRootHub@CHcd@@QAAPAVCRootHub@@PAV2@@Z 100027ac f   usbh_usb2com_common_topaz_v1:hcd.obj
 0001:000017d8       ?OpenPipe@CHcd@@QAAHIPBU_USB_ENDPOINT_DESCRIPTOR@@PAI@Z 100027d8 f   usbh_usb2com_common_topaz_v1:hcd.obj
 0001:00001860       ?ClosePipe@CHcd@@QAAHII@Z  10002860 f   usbh_usb2com_common_topaz_v1:hcd.obj
 0001:000018b8       ?IssueTransfer@CHcd@@QAAHIIP6AKPAX@Z0KPBXKKPBKK0K2PAK4PAH44@Z 100028b8 f   usbh_usb2com_common_topaz_v1:hcd.obj
 0001:000019ac       ?AbortTransfer@CHcd@@QAAHIIP6AKPAX@Z0PBX@Z 100029ac f   usbh_usb2com_common_topaz_v1:hcd.obj
 0001:00001a24       ?IsPipeHalted@CHcd@@QAAHIIPAH@Z 10002a24 f   usbh_usb2com_common_topaz_v1:hcd.obj
 0001:00001a8c       ?ResetPipe@CHcd@@QAAHII@Z  10002a8c f   usbh_usb2com_common_topaz_v1:hcd.obj
 0001:00001ae4       ?DisableDevice@CHcd@@UAAHIH@Z 10002ae4 f   usbh_usb2com_common_topaz_v1:hcd.obj
 0001:00001b3c       ?SuspendResume@CHcd@@UAAHIH@Z 10002b3c f   usbh_usb2com_common_topaz_v1:hcd.obj
 0001:00001b94       ??_ECHcd@@UAAPAXI@Z        10002b94 f i usbh_usb2com_common_topaz_v1:hcd.obj
 0001:00001b94       ??_GCHcd@@UAAPAXI@Z        10002b94 f i usbh_usb2com_common_topaz_v1:hcd.obj
 0001:00001bb8       ?CreateNewNode@CPhysMem@@AAAPAUtMEMLIST@@KKK@Z 10002bb8 f   usbh_usb2com_common_topaz_v1:cphysmem.obj
 0001:00001c34       ?FindFreeBlock@CPhysMem@@AAAPAUtMEMLIST@@KH@Z 10002c34 f   usbh_usb2com_common_topaz_v1:cphysmem.obj
 0001:00001ca0       ?AddNodeToFreeList@CPhysMem@@AAAHPAUtMEMLIST@@H@Z 10002ca0 f   usbh_usb2com_common_topaz_v1:cphysmem.obj
 0001:00001e34       ?FreeList@CPhysMem@@AAAHPAPAUtMEMLIST@@@Z 10002e34 f   usbh_usb2com_common_topaz_v1:cphysmem.obj
 0001:00001e80       ?AllocateSpecialMemory@CPhysMem@@QAAHKQAPAE@Z 10002e80 f   usbh_usb2com_common_topaz_v1:cphysmem.obj
 0001:00001ea0       ?FreeSpecialMemory@CPhysMem@@QAAXQAE@Z 10002ea0 f   usbh_usb2com_common_topaz_v1:cphysmem.obj
 0001:00001eac       ?AllocateMemory@CPhysMem@@QAAHKQAPAEKPAH@Z 10002eac f   usbh_usb2com_common_topaz_v1:cphysmem.obj
 0001:00002018       ?FreeMemory@CPhysMem@@QAAXQAEKK@Z 10003018 f   usbh_usb2com_common_topaz_v1:cphysmem.obj
 0001:000020fc       ?ReInit@CPhysMem@@QAAXXZ   100030fc f   usbh_usb2com_common_topaz_v1:cphysmem.obj
 0001:0000229c       ??1CPhysMem@@QAA@XZ        1000329c f   usbh_usb2com_common_topaz_v1:cphysmem.obj
 0001:00002304       ??0CPhysMem@@QAA@KKPAE0@Z  10003304 f   usbh_usb2com_common_topaz_v1:cphysmem.obj
 0001:00002470       ?WaitForAPIReadyWrapper@@YAKKK@Z 10003470 f i usbh_usb2com_common_topaz_v1:cdevice.obj
 0001:000024e0       ?CeCallUserProcWrapper@@YAHPBG0PAXK1KPAK@Z 100034e0 f i usbh_usb2com_common_topaz_v1:cdevice.obj
 0001:0000257c       ??0CDeviceGlobal@@QAA@XZ   1000357c f   usbh_usb2com_common_topaz_v1:cdevice.obj
 0001:000025dc       ?Initialize@CDeviceGlobal@@QAAHPAX@Z 100035dc f   usbh_usb2com_common_topaz_v1:cdevice.obj
 0001:000026bc       ?DeInitialize@CDeviceGlobal@@UAAXXZ 100036bc f   usbh_usb2com_common_topaz_v1:cdevice.obj
 0001:0000272c       ?ReserveAddress@CDeviceGlobal@@QAAHAAE@Z 1000372c f   usbh_usb2com_common_topaz_v1:cdevice.obj
 0001:000027b0       ?FreeAddress@CDeviceGlobal@@QAAXE@Z 100037b0 f   usbh_usb2com_common_topaz_v1:cdevice.obj
 0001:000027f0       ?TransferDoneCallbackSetEvent@CDevice@@KAKPAX@Z 100037f0 f   usbh_usb2com_common_topaz_v1:cdevice.obj
 0001:00002804       ??0CDevice@@QAA@EABU_USB_DEVICE_INFO@@HHEQAVCDeviceGlobal@@QAVCHub@@E@Z 10003804 f   usbh_usb2com_common_topaz_v1:cdevice.obj
 0001:00002884       ?ResumeNotification@CDevice@@UAAHXZ 10003884 f i usbh_usb2com_common_topaz_v1:cdevice.obj
 0001:0000288c       ?GetUSB2TT@CDevice@@UAAPAVCHub@@PAE0@Z 1000388c f   usbh_usb2com_common_topaz_v1:cdevice.obj
 0001:000028f4       ?DeleteUsbConfigurationStructure@CDevice@@QBAXAAU_NON_CONST_USB_CONFIGURATION@@@Z 100038f4 f   usbh_usb2com_common_topaz_v1:cdevice.obj
 0001:000029a0       ?AllocatePipeArray@CDevice@@IAAHXZ 100039a0 f   usbh_usb2com_common_topaz_v1:cdevice.obj
 0001:00002a68       ?SubHubTestModeEnable@CHub@@UAAHGG@Z 10003a68 f   usbh_usb2com_common_topaz_v1:cdevice.obj
 0001:00002a70       ?DisableDevice@CDevice@@UAA?AW4HCD_REQUEST_STATUS@@IH@Z 10003a70 f   usbh_usb2com_common_topaz_v1:cdevice.obj
 0001:00002aa0       ?SuspendResume@CDevice@@UAA?AW4HCD_REQUEST_STATUS@@IH@Z 10003aa0 f   usbh_usb2com_common_topaz_v1:cdevice.obj
 0001:00002b00       ?MessageBoxSpecial@CHub@@QAAHPAUHWND__@@PBGI@Z 10003b00 f   usbh_usb2com_common_topaz_v1:cdevice.obj
 0001:00002bcc       ?GetDescriptor@CHub@@IAAHQAVCPipeAbs@@EEEGPAX@Z 10003bcc f   usbh_usb2com_common_topaz_v1:cdevice.obj
 0001:00002d54       ?DetachDownstreamDeviceThread@CHub@@IAAKXZ 10003d54 f   usbh_usb2com_common_topaz_v1:cdevice.obj
 0001:00002dac       ?AllocateDeviceArray@CHub@@IAAHXZ 10003dac f   usbh_usb2com_common_topaz_v1:cdevice.obj
 0001:00002e80       ?HandleDetach@CHub@@UAAXXZ 10003e80 f   usbh_usb2com_common_topaz_v1:cdevice.obj
 0001:00002fe0       ?OpenPipe@CHub@@UAA?AW4HCD_REQUEST_STATUS@@IQBU_USB_ENDPOINT_DESCRIPTOR@@QAI@Z 10003fe0 f   usbh_usb2com_common_topaz_v1:cdevice.obj
 0001:0000306c       ?ClosePipe@CHub@@UAA?AW4HCD_REQUEST_STATUS@@II@Z 1000406c f   usbh_usb2com_common_topaz_v1:cdevice.obj
 0001:000030f0       ?IssueTransfer@CHub@@UAA?AW4HCD_REQUEST_STATUS@@IIQ6AKPAX@ZQAXKQBXKKQBKK2K3QAK5QAH55@Z 100040f0 f   usbh_usb2com_common_topaz_v1:cdevice.obj
 0001:00003200       ?AbortTransfer@CHub@@UAA?AW4HCD_REQUEST_STATUS@@IIQ6AKPAX@ZQAXQBX@Z 10004200 f   usbh_usb2com_common_topaz_v1:cdevice.obj
 0001:000032a4       ?IsPipeHalted@CHub@@UAA?AW4HCD_REQUEST_STATUS@@IIQAH@Z 100042a4 f   usbh_usb2com_common_topaz_v1:cdevice.obj
 0001:00003330       ?ResetPipe@CHub@@UAA?AW4HCD_REQUEST_STATUS@@II@Z 10004330 f   usbh_usb2com_common_topaz_v1:cdevice.obj
 0001:000033b4       ?DisableDevice@CHub@@UAA?AW4HCD_REQUEST_STATUS@@IH@Z 100043b4 f   usbh_usb2com_common_topaz_v1:cdevice.obj
 0001:000033f8       ?SuspendResume@CHub@@UAA?AW4HCD_REQUEST_STATUS@@IH@Z 100043f8 f   usbh_usb2com_common_topaz_v1:cdevice.obj
 0001:00003490       ?SuspendResumeOffStreamDevice@CHub@@UAAHIH@Z 10004490 f   usbh_usb2com_common_topaz_v1:cdevice.obj
 0001:00003548       ?PowerAllHubPorts@CRootHub@@EAAHXZ 10004548 f   usbh_usb2com_common_topaz_v1:cdevice.obj
 0001:00003550       ?WaitForPortStatusChange@CRootHub@@EAAHAAEAAU_USB_HUB_AND_PORT_STATUS@@PAK@Z 10004550 f   usbh_usb2com_common_topaz_v1:cdevice.obj
 0001:000037d0       ?GetStatus@CRootHub@@EAAHEAAU_USB_HUB_AND_PORT_STATUS@@PAK@Z 100047d0 f   usbh_usb2com_common_topaz_v1:cdevice.obj
 0001:000037e8       ?ResetAndEnablePort@CRootHub@@EAAHE@Z 100047e8 f   usbh_usb2com_common_topaz_v1:cdevice.obj
 0001:00003800       ?DisablePort@CRootHub@@EAAXE@Z 10004800 f   usbh_usb2com_common_topaz_v1:cdevice.obj
 0001:00003818       ?SetOrClearFeature@CRootHub@@EAAHGEG@Z 10004818 f   usbh_usb2com_common_topaz_v1:cdevice.obj
 0001:00003834       ?SetOrClearRemoteWakup@CRootHub@@EAAHH@Z 10004834 f   usbh_usb2com_common_topaz_v1:cdevice.obj
 0001:0000383c       ?SubHubTestModeEnable@CRootHub@@UAAHGG@Z 1000483c f   usbh_usb2com_common_topaz_v1:cdevice.obj
 0001:00003924       ?SubHubTestModeEnable@CExternalHub@@UAAHGG@Z 10004924 f   usbh_usb2com_common_topaz_v1:cdevice.obj
 0001:00003ab0       ?PowerAllHubPorts@CExternalHub@@EAAHXZ 10004ab0 f   usbh_usb2com_common_topaz_v1:cdevice.obj
 0001:00003b80       ?GetStatusChangeBitmap@CExternalHub@@AAAHAAK@Z 10004b80 f   usbh_usb2com_common_topaz_v1:cdevice.obj
 0001:00003ce8       ?WaitForPortStatusChange@CExternalHub@@EAAHAAEAAU_USB_HUB_AND_PORT_STATUS@@PAK@Z 10004ce8 f   usbh_usb2com_common_topaz_v1:cdevice.obj
 0001:00003e0c       ?GetStatus@CExternalHub@@EAAHEAAU_USB_HUB_AND_PORT_STATUS@@PAK@Z 10004e0c f   usbh_usb2com_common_topaz_v1:cdevice.obj
 0001:00003f58       ?ResetAndEnablePort@CExternalHub@@EAAHE@Z 10004f58 f   usbh_usb2com_common_topaz_v1:cdevice.obj
 0001:00004084       ?DisablePort@CExternalHub@@EAAXE@Z 10005084 f   usbh_usb2com_common_topaz_v1:cdevice.obj
 0001:000040b4       ?SetOrClearFeature@CExternalHub@@EAAHGEG@Z 100050b4 f   usbh_usb2com_common_topaz_v1:cdevice.obj
 0001:000041fc       ?SetOrClearRemoteWakup@CExternalHub@@EAAHH@Z 100051fc f   usbh_usb2com_common_topaz_v1:cdevice.obj
 0001:00004344       ?EnterOperationalState@CFunction@@UAAHQAVCPipeAbs@@@Z 10005344 f   usbh_usb2com_common_topaz_v1:cdevice.obj
 0001:00004448       ?OpenPipe@CFunction@@UAA?AW4HCD_REQUEST_STATUS@@IQBU_USB_ENDPOINT_DESCRIPTOR@@QAI@Z 10005448 f   usbh_usb2com_common_topaz_v1:cdevice.obj
 0001:00004730       ?ClosePipe@CFunction@@UAA?AW4HCD_REQUEST_STATUS@@II@Z 10005730 f   usbh_usb2com_common_topaz_v1:cdevice.obj
 0001:000047c4       ?IssueTransfer@CFunction@@UAA?AW4HCD_REQUEST_STATUS@@IIQ6AKPAX@ZQAXKQBXKKQBKK2K3QAK5QAH55@Z 100057c4 f   usbh_usb2com_common_topaz_v1:cdevice.obj
 0001:000048e0       ?AbortTransfer@CFunction@@UAA?AW4HCD_REQUEST_STATUS@@IIQ6AKPAX@ZQAXQBX@Z 100058e0 f   usbh_usb2com_common_topaz_v1:cdevice.obj
 0001:0000495c       ?IsPipeHalted@CFunction@@UAA?AW4HCD_REQUEST_STATUS@@IIQAH@Z 1000595c f   usbh_usb2com_common_topaz_v1:cdevice.obj
 0001:000049e4       ?HandleDetach@CFunction@@EAAXXZ 100059e4 f   usbh_usb2com_common_topaz_v1:cdevice.obj
 0001:00004b5c       ?SetOrClearFeature@CFunction@@AAAHEGEG@Z 10005b5c f   usbh_usb2com_common_topaz_v1:cdevice.obj
 0001:00004c88       ??1CDeviceGlobal@@UAA@XZ   10005c88 f   usbh_usb2com_common_topaz_v1:cdevice.obj
 0001:00004cbc       ??1CDevice@@UAA@XZ         10005cbc f   usbh_usb2com_common_topaz_v1:cdevice.obj
 0001:00004d50       ?CreateUsbConfigurationStructure@CDevice@@QBAHAAU_NON_CONST_USB_CONFIGURATION@@QAEI@Z 10005d50 f   usbh_usb2com_common_topaz_v1:cdevice.obj
 0001:000050cc       ??0CHub@@QAA@EABU_USB_DEVICE_INFO@@HHEABU_USB_HUB_DESCRIPTOR@@QAVCHcd@@QAV0@E@Z 100060cc f   usbh_usb2com_common_topaz_v1:cdevice.obj
 0001:000051f8       ?ResumeNotification@CHub@@UAAHXZ 100061f8 f i usbh_usb2com_common_topaz_v1:cdevice.obj
 0001:00005210       ??1CHub@@UAA@XZ            10006210 f   usbh_usb2com_common_topaz_v1:cdevice.obj
 0001:0000529c       ?DetachDownstreamDeviceThreadStub@CHub@@KAKPAX@Z 1000629c f   usbh_usb2com_common_topaz_v1:cdevice.obj
 0001:000052a0       ?DetachDevice@CHub@@IAAXE@Z 100062a0 f   usbh_usb2com_common_topaz_v1:cdevice.obj
 0001:0000540c       ??0CRootHub@@QAA@ABU_USB_DEVICE_INFO@@HHABU_USB_HUB_DESCRIPTOR@@QAVCHcd@@@Z 1000640c f   usbh_usb2com_common_topaz_v1:cdevice.obj
 0001:00005468       ?GetDeviceTypeInt@CRootHub@@EBA?BKXZ 10006468 f i usbh_usb2com_common_topaz_v1:cdevice.obj
 0001:00005470       ??0CExternalHub@@QAA@EABU_USB_DEVICE_INFO@@HHEABU_USB_HUB_DESCRIPTOR@@QAVCHcd@@QAVCHub@@E@Z 10006470 f   usbh_usb2com_common_topaz_v1:cdevice.obj
 0001:000054c8       ?GetDeviceTypeInt@CExternalHub@@EBA?BKXZ 100064c8 f i usbh_usb2com_common_topaz_v1:cdevice.obj
 0001:000054d0       ??0CFunction@@QAA@EABU_USB_DEVICE_INFO@@HHEQAVCHcd@@QAVCHub@@E@Z 100064d0 f   usbh_usb2com_common_topaz_v1:cdevice.obj
 0001:00005534       ?GetDeviceTypeInt@CFunction@@EBA?BKXZ 10006534 f i usbh_usb2com_common_topaz_v1:cdevice.obj
 0001:0000553c       ?ResetPipe@CFunction@@UAA?AW4HCD_REQUEST_STATUS@@II@Z 1000653c f   usbh_usb2com_common_topaz_v1:cdevice.obj
 0001:000055ec       ??_ECDeviceGlobal@@UAAPAXI@Z 100065ec f i usbh_usb2com_common_topaz_v1:cdevice.obj
 0001:000055ec       ??_GCDeviceGlobal@@UAAPAXI@Z 100065ec f i usbh_usb2com_common_topaz_v1:cdevice.obj
 0001:00005610       ??_GCDevice@@UAAPAXI@Z     10006610 f i usbh_usb2com_common_topaz_v1:cdevice.obj
 0001:00005610       ??_ECDevice@@UAAPAXI@Z     10006610 f i usbh_usb2com_common_topaz_v1:cdevice.obj
 0001:00005634       ??_ECHub@@UAAPAXI@Z        10006634 f i usbh_usb2com_common_topaz_v1:cdevice.obj
 0001:00005634       ??_GCHub@@UAAPAXI@Z        10006634 f i usbh_usb2com_common_topaz_v1:cdevice.obj
 0001:00005660       ?AttachDevice@CHub@@IAAXEHH@Z 10006660 f   usbh_usb2com_common_topaz_v1:cdevice.obj
 0001:00006304       ?DisableOffStreamDevice@CHub@@UAAHIH@Z 10007304 f   usbh_usb2com_common_topaz_v1:cdevice.obj
 0001:000063e0       ??_GCRootHub@@UAAPAXI@Z    100073e0 f i usbh_usb2com_common_topaz_v1:cdevice.obj
 0001:000063e0       ??_ECRootHub@@UAAPAXI@Z    100073e0 f i usbh_usb2com_common_topaz_v1:cdevice.obj
 0001:00006410       ??_GCExternalHub@@UAAPAXI@Z 10007410 f i usbh_usb2com_common_topaz_v1:cdevice.obj
 0001:00006410       ??_ECExternalHub@@UAAPAXI@Z 10007410 f i usbh_usb2com_common_topaz_v1:cdevice.obj
 0001:00006440       ??_GCFunction@@UAAPAXI@Z   10007440 f i usbh_usb2com_common_topaz_v1:cdevice.obj
 0001:00006440       ??_ECFunction@@UAAPAXI@Z   10007440 f i usbh_usb2com_common_topaz_v1:cdevice.obj
 0001:00006470       ?HubStatusChangeThread@CHub@@AAAKXZ 10007470 f   usbh_usb2com_common_topaz_v1:cdevice.obj
 0001:000069f4       ?HubStatusChangeThreadStub@CHub@@KAKPAX@Z 100079f4 f   usbh_usb2com_common_topaz_v1:cdevice.obj
 0001:000069f8       ?EnterOperationalState@CRootHub@@UAAHQAVCPipeAbs@@@Z 100079f8 f   usbh_usb2com_common_topaz_v1:cdevice.obj
 0001:00006ab8       ?EnterOperationalState@CExternalHub@@UAAHQAVCPipeAbs@@@Z 10007ab8 f   usbh_usb2com_common_topaz_v1:cdevice.obj
 0001:00006c5c       ?EnterCritSec_Ex@CritSec_Ex@@QAA?AW4e_CritSec_Status@@K@Z 10007c5c f   usbh_usb2com_common_topaz_v1:sync.obj
 0001:00006d7c       ?LeaveCritSec_Ex@CritSec_Ex@@QAAXXZ 10007d7c f   usbh_usb2com_common_topaz_v1:sync.obj
 0001:00006db8       ?Initialize@CritSec_Ex@@QAAXXZ 10007db8 f   usbh_usb2com_common_topaz_v1:sync.obj
 0001:00006de8       ?PrepareDeleteCritSec_Ex@CritSec_Ex@@QAAXXZ 10007de8 f   usbh_usb2com_common_topaz_v1:sync.obj
 0001:00006e34       ??1CritSec_Ex@@QAA@XZ      10007e34 f   usbh_usb2com_common_topaz_v1:sync.obj
 0001:00006e9c       ??0Countdown@@QAA@K@Z      10007e9c f   usbh_usb2com_common_topaz_v1:sync.obj
 0001:00006ee4       ?IncrCountdown@Countdown@@QAAHXZ 10007ee4 f   usbh_usb2com_common_topaz_v1:sync.obj
 0001:00006f30       ?DecrCountdown@Countdown@@QAAXXZ 10007f30 f   usbh_usb2com_common_topaz_v1:sync.obj
 0001:00006f60       ?WaitForCountdown@Countdown@@QAAXH@Z 10007f60 f   usbh_usb2com_common_topaz_v1:sync.obj
 0001:00006f94       ??1Countdown@@QAA@XZ       10007f94 f   usbh_usb2com_common_topaz_v1:sync.obj
 0001:00006fb8       ??0CritSec_Ex@@QAA@XZ      10007fb8 f   usbh_usb2com_common_topaz_v1:sync.obj
 0001:00007008       ??0CEhcd@@QAA@PAXPAVCPhysMem@@PBGRAEKK@Z 10008008 f   usbh_ehcdmdd_common_topaz_v1:cehcd.obj
 0001:00007068       ?SignalCheckForDoneTransfers@CHW@@UAAXXZ 10008068 f i usbh_ehcdmdd_common_topaz_v1:cehcd.obj
 0001:00007070       ?GetForceReAttach@CHW@@UAAKXZ 10008070 f i usbh_ehcdmdd_common_topaz_v1:cehcd.obj
 0001:00007078       ?SetForceReAttach@CHW@@UAAXK@Z 10008078 f i usbh_ehcdmdd_common_topaz_v1:cehcd.obj
 0001:00007080       ?GetCapability@CHW@@UAAKXZ 10008080 f i usbh_ehcdmdd_common_topaz_v1:cehcd.obj
 0001:00007088       ?SignalHubStatusChange@CHW@@UAAXXZ 10008088 f i usbh_ehcdmdd_common_topaz_v1:cehcd.obj
 0001:000070a4       ?AddedTt@CEhcd@@UAAHEE@Z   100080a4 f i usbh_ehcdmdd_common_topaz_v1:cehcd.obj
 0001:000070ac       ?DeleteTt@CEhcd@@UAAHEE@Z  100080ac f i usbh_ehcdmdd_common_topaz_v1:cehcd.obj
 0001:000070b4       ??1CEhcd@@UAA@XZ           100080b4 f   usbh_ehcdmdd_common_topaz_v1:cehcd.obj
 0001:00007118       ?DeviceDeInitialize@CEhcd@@UAAXXZ 10008118 f   usbh_ehcdmdd_common_topaz_v1:cehcd.obj
 0001:00007178       ?DeviceInitialize@CEhcd@@UAAHXZ 10008178 f   usbh_ehcdmdd_common_topaz_v1:cehcd.obj
 0001:000072fc       ?CreateHCDObject@@YAPAVCHcd@@PAXPAVCPhysMem@@KPBGRAEK@Z 100082fc f   usbh_ehcdmdd_common_topaz_v1:cehcd.obj
 0001:0000735c       ??_GCEhcd@@UAAPAXI@Z       1000835c f i usbh_ehcdmdd_common_topaz_v1:cehcd.obj
 0001:0000735c       ??_ECEhcd@@UAAPAXI@Z       1000835c f i usbh_ehcdmdd_common_topaz_v1:cehcd.obj
 0001:00007380       ??0CQTransfer@@QAA@QAVCPipe@@QAVCPhysMem@@PAUSTRANSFER@@@Z 10008380 f i usbh_ehcdmdd_common_topaz_v1:cpipe.obj
 0001:000073a8       ??_GCQTransfer@@UAAPAXI@Z  100083a8 f i usbh_ehcdmdd_common_topaz_v1:cpipe.obj
 0001:000073a8       ??_ECQTransfer@@UAAPAXI@Z  100083a8 f i usbh_ehcdmdd_common_topaz_v1:cpipe.obj
 0001:000073cc       ?ChangeMaxPacketSize@CPipeAbs@@UAAXG@Z 100083cc f i usbh_ehcdmdd_common_topaz_v1:cpipe.obj
 0001:000073d0       ??_GCPipeAbs@@UAAPAXI@Z    100083d0 f i usbh_ehcdmdd_common_topaz_v1:cpipe.obj
 0001:000073d0       ??_ECPipeAbs@@UAAPAXI@Z    100083d0 f i usbh_ehcdmdd_common_topaz_v1:cpipe.obj
 0001:000073f4       ??0CPipe@@QAA@QBU_USB_ENDPOINT_DESCRIPTOR@@HHEEEQAVCEhcd@@@Z 100083f4 f   usbh_ehcdmdd_common_topaz_v1:cpipe.obj
 0001:00007488       ??1CPipe@@UAA@XZ           10008488 f   usbh_ehcdmdd_common_topaz_v1:cpipe.obj
 0001:000074b0       ?GetCPhysMem@CPipe@@UAAPAVCPhysMem@@XZ 100084b0 f   usbh_ehcdmdd_common_topaz_v1:cpipe.obj
 0001:000074bc       ?IsPipeHalted@CPipe@@UAA?AW4HCD_REQUEST_STATUS@@QAH@Z 100084bc f   usbh_ehcdmdd_common_topaz_v1:cpipe.obj
 0001:000074ec       ?ClearHaltedFlag@CPipe@@UAAXXZ 100084ec f   usbh_ehcdmdd_common_topaz_v1:cpipe.obj
 0001:00007510       ??0CQueuedPipe@@QAA@QBU_USB_ENDPOINT_DESCRIPTOR@@HHEEEQAVCEhcd@@@Z 10008510 f   usbh_ehcdmdd_common_topaz_v1:cpipe.obj
 0001:00007568       ??1CQueuedPipe@@UAA@XZ     10008568 f   usbh_ehcdmdd_common_topaz_v1:cpipe.obj
 0001:000075b4       ?ClearHaltedFlag@CQueuedPipe@@UAAXXZ 100085b4 f   usbh_ehcdmdd_common_topaz_v1:cpipe.obj
 0001:000075f0       ?IssueTransfer@CQueuedPipe@@UAA?AW4HCD_REQUEST_STATUS@@EQ6AKPAX@ZQAXKQBXKKQBKK2K3QAK5QAH55@Z 100085f0 f   usbh_ehcdmdd_common_topaz_v1:cpipe.obj
 0001:00007808       ?GetPipeType@CBulkPipe@@UBAPBGXZ 10008808 f i usbh_ehcdmdd_common_topaz_v1:cpipe.obj
 0001:00007814       ?RemoveQHeadFromQueue@CBulkPipe@@MAAHXZ 10008814 f   usbh_ehcdmdd_common_topaz_v1:cpipe.obj
 0001:00007834       ?InsertQHeadToQueue@CBulkPipe@@MAAHXZ 10008834 f   usbh_ehcdmdd_common_topaz_v1:cpipe.obj
 0001:00007858       ?AreTransferParametersValid@CBulkPipe@@EBAHPBUSTRANSFER@@@Z 10008858 f   usbh_ehcdmdd_common_topaz_v1:cpipe.obj
 0001:000078c4       ?GetPipeType@CControlPipe@@UBAPBGXZ 100088c4 f i usbh_ehcdmdd_common_topaz_v1:cpipe.obj
 0001:000078d0       ?RemoveQHeadFromQueue@CControlPipe@@MAAHXZ 100088d0 f   usbh_ehcdmdd_common_topaz_v1:cpipe.obj
 0001:000078f0       ?InsertQHeadToQueue@CControlPipe@@MAAHXZ 100088f0 f   usbh_ehcdmdd_common_topaz_v1:cpipe.obj
 0001:00007914       ?AreTransferParametersValid@CControlPipe@@EBAHPBUSTRANSFER@@@Z 10008914 f   usbh_ehcdmdd_common_topaz_v1:cpipe.obj
 0001:000079b8       ??0CInterruptPipe@@QAA@QBU_USB_ENDPOINT_DESCRIPTOR@@HHEEEQAVCEhcd@@@Z 100089b8 f   usbh_ehcdmdd_common_topaz_v1:cpipe.obj
 0001:00007b64       ?GetPipeType@CInterruptPipe@@UBAPBGXZ 10008b64 f i usbh_ehcdmdd_common_topaz_v1:cpipe.obj
 0001:00007b74       ?RemoveQHeadFromQueue@CInterruptPipe@@MAAHXZ 10008b74 f i usbh_ehcdmdd_common_topaz_v1:cpipe.obj
 0001:00007b7c       ?InsertQHeadToQueue@CInterruptPipe@@MAAHXZ 10008b7c f i usbh_ehcdmdd_common_topaz_v1:cpipe.obj
 0001:00007b84       ?AreTransferParametersValid@CInterruptPipe@@EBAHPBUSTRANSFER@@@Z 10008b84 f   usbh_ehcdmdd_common_topaz_v1:cpipe.obj
 0001:00007bf0       ??0CIsochronousPipe@@QAA@QBU_USB_ENDPOINT_DESCRIPTOR@@HHEEEQAVCEhcd@@@Z 10008bf0 f   usbh_ehcdmdd_common_topaz_v1:cpipe.obj
 0001:00007eb8       ?GetPipeType@CIsochronousPipe@@UBAPBGXZ 10008eb8 f i usbh_ehcdmdd_common_topaz_v1:cpipe.obj
 0001:00007ec8       ?StopTransfers@CIsochronousPipe@@UAAXXZ 10008ec8 f i usbh_ehcdmdd_common_topaz_v1:cpipe.obj
 0001:00007ecc       ?AllocateCITD@CIsochronousPipe@@QAAPAVCITD@@PAVCITransfer@@@Z 10008ecc f   usbh_ehcdmdd_common_topaz_v1:cpipe.obj
 0001:00007f48       ?AllocateCSITD@CIsochronousPipe@@QAAPAVCSITD@@PAVCSITransfer@@PAV2@@Z 10008f48 f   usbh_ehcdmdd_common_topaz_v1:cpipe.obj
 0001:00007fcc       ?OpenPipe@CIsochronousPipe@@UAA?AW4HCD_REQUEST_STATUS@@XZ 10008fcc f   usbh_ehcdmdd_common_topaz_v1:cpipe.obj
 0001:0000803c       ?ClosePipe@CIsochronousPipe@@UAA?AW4HCD_REQUEST_STATUS@@XZ 1000903c f   usbh_ehcdmdd_common_topaz_v1:cpipe.obj
 0001:000080b8       ?AbortTransfer@CIsochronousPipe@@UAA?AW4HCD_REQUEST_STATUS@@Q6AKPAX@ZQAXPBX@Z 100090b8 f   usbh_ehcdmdd_common_topaz_v1:cpipe.obj
 0001:000081c8       ?IssueTransfer@CIsochronousPipe@@UAA?AW4HCD_REQUEST_STATUS@@EQ6AKPAX@ZQAXKQBXKKQBKK2K3QAK5QAH55@Z 100091c8 f   usbh_ehcdmdd_common_topaz_v1:cpipe.obj
 0001:000084d8       ?ScheduleTransfer@CIsochronousPipe@@UAA?AW4HCD_REQUEST_STATUS@@XZ 100094d8 f   usbh_ehcdmdd_common_topaz_v1:cpipe.obj
 0001:00008548       ?CheckForDoneTransfers@CIsochronousPipe@@UAAHXZ 10009548 f   usbh_ehcdmdd_common_topaz_v1:cpipe.obj
 0001:00008634       ?AreTransferParametersValid@CIsochronousPipe@@EBAHPBUSTRANSFER@@@Z 10009634 f   usbh_ehcdmdd_common_topaz_v1:cpipe.obj
 0001:00008774       ?CreateBulkPipe@@YAPAVCPipeAbs@@QBU_USB_ENDPOINT_DESCRIPTOR@@HHEEEQAVCHcd@@@Z 10009774 f   usbh_ehcdmdd_common_topaz_v1:cpipe.obj
 0001:000087ec       ?CreateControlPipe@@YAPAVCPipeAbs@@QBU_USB_ENDPOINT_DESCRIPTOR@@HHEEEQAVCHcd@@@Z 100097ec f   usbh_ehcdmdd_common_topaz_v1:cpipe.obj
 0001:00008864       ?CreateInterruptPipe@@YAPAVCPipeAbs@@QBU_USB_ENDPOINT_DESCRIPTOR@@HHEEEQAVCHcd@@@Z 10009864 f   usbh_ehcdmdd_common_topaz_v1:cpipe.obj
 0001:000088cc       ?CreateIsochronousPipe@@YAPAVCPipeAbs@@QBU_USB_ENDPOINT_DESCRIPTOR@@HHEEEQAVCHcd@@@Z 100098cc f   usbh_ehcdmdd_common_topaz_v1:cpipe.obj
 0001:00008934       ??_ECPipe@@UAAPAXI@Z       10009934 f i usbh_ehcdmdd_common_topaz_v1:cpipe.obj
 0001:00008934       ??_GCPipe@@UAAPAXI@Z       10009934 f i usbh_ehcdmdd_common_topaz_v1:cpipe.obj
 0001:00008970       ??_GCQueuedPipe@@UAAPAXI@Z 10009970 f i usbh_ehcdmdd_common_topaz_v1:cpipe.obj
 0001:00008970       ??_ECQueuedPipe@@UAAPAXI@Z 10009970 f i usbh_ehcdmdd_common_topaz_v1:cpipe.obj
 0001:0000899c       ?AbortTransfer@CQueuedPipe@@UAA?AW4HCD_REQUEST_STATUS@@Q6AKPAX@ZQAXPBX@Z 1000999c f   usbh_ehcdmdd_common_topaz_v1:cpipe.obj
 0001:00008b70       ?AbortQueue@CQueuedPipe@@IAAXXZ 10009b70 f   usbh_ehcdmdd_common_topaz_v1:cpipe.obj
 0001:00008c80       ?StopTransfers@CQueuedPipe@@UAAXXZ 10009c80 f   usbh_ehcdmdd_common_topaz_v1:cpipe.obj
 0001:00008c94       ?ScheduleTransfer@CQueuedPipe@@UAA?AW4HCD_REQUEST_STATUS@@XZ 10009c94 f   usbh_ehcdmdd_common_topaz_v1:cpipe.obj
 0001:00008d54       ?CheckForDoneTransfers@CQueuedPipe@@UAAHXZ 10009d54 f   usbh_ehcdmdd_common_topaz_v1:cpipe.obj
 0001:00008e58       ?OpenPipe@CBulkPipe@@UAA?AW4HCD_REQUEST_STATUS@@XZ 10009e58 f   usbh_ehcdmdd_common_topaz_v1:cpipe.obj
 0001:00008f1c       ?ClosePipe@CBulkPipe@@UAA?AW4HCD_REQUEST_STATUS@@XZ 10009f1c f   usbh_ehcdmdd_common_topaz_v1:cpipe.obj
 0001:00008f94       ?OpenPipe@CControlPipe@@UAA?AW4HCD_REQUEST_STATUS@@XZ 10009f94 f   usbh_ehcdmdd_common_topaz_v1:cpipe.obj
 0001:00009070       ?ClosePipe@CControlPipe@@UAA?AW4HCD_REQUEST_STATUS@@XZ 1000a070 f   usbh_ehcdmdd_common_topaz_v1:cpipe.obj
 0001:000090e8       ?IssueTransfer@CControlPipe@@UAA?AW4HCD_REQUEST_STATUS@@EQ6AKPAX@ZQAXKQBXKKQBKK2K3QAK5QAH55@Z 1000a0e8 f   usbh_ehcdmdd_common_topaz_v1:cpipe.obj
 0001:00009214       ?ChangeMaxPacketSize@CControlPipe@@UAAXG@Z 1000a214 f   usbh_ehcdmdd_common_topaz_v1:cpipe.obj
 0001:000092a8       ?OpenPipe@CInterruptPipe@@UAA?AW4HCD_REQUEST_STATUS@@XZ 1000a2a8 f   usbh_ehcdmdd_common_topaz_v1:cpipe.obj
 0001:000093c8       ?ClosePipe@CInterruptPipe@@UAA?AW4HCD_REQUEST_STATUS@@XZ 1000a3c8 f   usbh_ehcdmdd_common_topaz_v1:cpipe.obj
 0001:00009444       ?FreeCITD@CIsochronousPipe@@QAAXPAVCITD@@@Z 1000a444 f   usbh_ehcdmdd_common_topaz_v1:cpipe.obj
 0001:00009490       ?FreeCSITD@CIsochronousPipe@@QAAXPAVCSITD@@@Z 1000a490 f   usbh_ehcdmdd_common_topaz_v1:cpipe.obj
 0001:000094dc       ??1CInterruptPipe@@UAA@XZ  1000a4dc f   usbh_ehcdmdd_common_topaz_v1:cpipe.obj
 0001:00009524       ??1CIsochronousPipe@@UAA@XZ 1000a524 f   usbh_ehcdmdd_common_topaz_v1:cpipe.obj
 0001:00009640       ??_ECBulkPipe@@UAAPAXI@Z   1000a640 f i usbh_ehcdmdd_common_topaz_v1:cpipe.obj
 0001:00009640       ??_GCBulkPipe@@UAAPAXI@Z   1000a640 f i usbh_ehcdmdd_common_topaz_v1:cpipe.obj
 0001:00009678       ??_ECControlPipe@@UAAPAXI@Z 1000a678 f i usbh_ehcdmdd_common_topaz_v1:cpipe.obj
 0001:00009678       ??_GCControlPipe@@UAAPAXI@Z 1000a678 f i usbh_ehcdmdd_common_topaz_v1:cpipe.obj
 0001:000096b0       ??_ECInterruptPipe@@UAAPAXI@Z 1000a6b0 f i usbh_ehcdmdd_common_topaz_v1:cpipe.obj
 0001:000096b0       ??_GCInterruptPipe@@UAAPAXI@Z 1000a6b0 f i usbh_ehcdmdd_common_topaz_v1:cpipe.obj
 0001:000096d4       ??_ECIsochronousPipe@@UAAPAXI@Z 1000a6d4 f i usbh_ehcdmdd_common_topaz_v1:cpipe.obj
 0001:000096d4       ??_GCIsochronousPipe@@UAAPAXI@Z 1000a6d4 f i usbh_ehcdmdd_common_topaz_v1:cpipe.obj
 0001:000096f8       ??0TransactionTrasnlate@@QAA@EEPAV0@@Z 1000a6f8 f   usbh_ehcdmdd_common_topaz_v1:usb2lib.obj
 0001:00009734       ??1TransactionTrasnlate@@QAA@XZ 1000a734 f   usbh_ehcdmdd_common_topaz_v1:usb2lib.obj
 0001:00009768       ?FindBestTimeSlot@TransactionTrasnlate@@AAAHGGPAU_ENDPOINTBUGETLIST@@PAK@Z 1000a768 f   usbh_ehcdmdd_common_topaz_v1:usb2lib.obj
 0001:000097b8       ?InsertEp@TransactionTrasnlate@@AAAHKPAU_EndpointBuget@@@Z 1000a7b8 f   usbh_ehcdmdd_common_topaz_v1:usb2lib.obj
 0001:000098a4       ?RemoveEp@TransactionTrasnlate@@AAAHKPAU_EndpointBuget@@@Z 1000a8a4 f   usbh_ehcdmdd_common_topaz_v1:usb2lib.obj
 0001:0000995c       ??0USB2lib@@QAA@XZ         1000a95c f   usbh_ehcdmdd_common_topaz_v1:usb2lib.obj
 0001:000099b8       ?DeleteTt@USB2lib@@QAAHEE@Z 1000a9b8 f   usbh_ehcdmdd_common_topaz_v1:usb2lib.obj
 0001:00009a44       ?GetTT@USB2lib@@QAAPAVTransactionTrasnlate@@EE@Z 1000aa44 f   usbh_ehcdmdd_common_topaz_v1:usb2lib.obj
 0001:00009a94       ?Compute_nonsplit_overhead@USB2lib@@AAAHPAU_EndpointBuget@@@Z 1000aa94 f   usbh_ehcdmdd_common_topaz_v1:usb2lib.obj
 0001:00009b04       ?ConvertBtoHFrame@USB2lib@@AAAXEEPAE0@Z 1000ab04 f   usbh_ehcdmdd_common_topaz_v1:usb2lib.obj
 0001:00009b44       ?AddedEp@TransactionTrasnlate@@QAAHPAU_EndpointBuget@@@Z 1000ab44 f   usbh_ehcdmdd_common_topaz_v1:usb2lib.obj
 0001:00009d60       ?DeletedEp@TransactionTrasnlate@@QAAHPAU_EndpointBuget@@@Z 1000ad60 f   usbh_ehcdmdd_common_topaz_v1:usb2lib.obj
 0001:00009dd4       ??1USB2lib@@QAA@XZ         1000add4 f   usbh_ehcdmdd_common_topaz_v1:usb2lib.obj
 0001:00009e20       ?AddedTt@USB2lib@@QAAHEE@Z 1000ae20 f   usbh_ehcdmdd_common_topaz_v1:usb2lib.obj
 0001:00009e98       ?AllocUsb2BusTime@USB2lib@@QAAHEEPAU_EndpointBuget@@@Z 1000ae98 f   usbh_ehcdmdd_common_topaz_v1:usb2lib.obj
 0001:0000a16c       ?FreeUsb2BusTime@USB2lib@@QAAXEEPAU_EndpointBuget@@@Z 1000b16c f   usbh_ehcdmdd_common_topaz_v1:usb2lib.obj
 0001:0000a220       ?GetSMASK@USB2lib@@QAAEPAU_EndpointBuget@@@Z 1000b220 f   usbh_ehcdmdd_common_topaz_v1:usb2lib.obj
 0001:0000a29c       ?GetCMASK@USB2lib@@QAAEPAU_EndpointBuget@@@Z 1000b29c f   usbh_ehcdmdd_common_topaz_v1:usb2lib.obj
 0001:0000a38c       ?SetNextPointer@CNextLinkPointer@@QAAHKW4NEXTLINKTYPE@@H@Z 1000b38c f i usbh_ehcdmdd_common_topaz_v1:chw.obj
 0001:0000a410       ??0CRegistryEdit@@QAA@PAUHKEY__@@PBG@Z 1000b410 f i usbh_ehcdmdd_common_topaz_v1:chw.obj
 0001:0000a45c       ?GetRegValue@CRegistryEdit@@QAAHPBGPAEK@Z 1000b45c f i usbh_ehcdmdd_common_topaz_v1:chw.obj
 0001:0000a4ac       ??0CDummyPipe@@QAA@QAVCPhysMem@@@Z 1000b4ac f   usbh_ehcdmdd_common_topaz_v1:chw.obj
 0001:0000a50c       ?IssueTransfer@CDummyPipe@@UAA?AW4HCD_REQUEST_STATUS@@EQ6AKPAX@ZQAXKQBXKKQBKK2K3QAK5QAH55@Z 1000b50c f i usbh_ehcdmdd_common_topaz_v1:chw.obj
 0001:0000a514       ?OpenPipe@CDummyPipe@@UAA?AW4HCD_REQUEST_STATUS@@XZ 1000b514 f i usbh_ehcdmdd_common_topaz_v1:chw.obj
 0001:0000a51c       ?ClosePipe@CDummyPipe@@UAA?AW4HCD_REQUEST_STATUS@@XZ 1000b51c f i usbh_ehcdmdd_common_topaz_v1:chw.obj
 0001:0000a524       ?IsPipeHalted@CDummyPipe@@UAA?AW4HCD_REQUEST_STATUS@@QAH@Z 1000b524 f i usbh_ehcdmdd_common_topaz_v1:chw.obj
 0001:0000a52c       ?ClearHaltedFlag@CDummyPipe@@UAAXXZ 1000b52c f i usbh_ehcdmdd_common_topaz_v1:chw.obj
 0001:0000a530       ?StopTransfers@CDummyPipe@@UAAXXZ 1000b530 f i usbh_ehcdmdd_common_topaz_v1:chw.obj
 0001:0000a534       ?AbortTransfer@CDummyPipe@@UAA?AW4HCD_REQUEST_STATUS@@Q6AKPAX@ZQAXPBX@Z 1000b534 f i usbh_ehcdmdd_common_topaz_v1:chw.obj
 0001:0000a53c       ?GetCPhysMem@CDummyPipe@@UAAPAVCPhysMem@@XZ 1000b53c f i usbh_ehcdmdd_common_topaz_v1:chw.obj
 0001:0000a544       ?ScheduleTransfer@CDummyPipe@@EAA?AW4HCD_REQUEST_STATUS@@XZ 1000b544 f i usbh_ehcdmdd_common_topaz_v1:chw.obj
 0001:0000a54c       ?GetPipeType@CDummyPipe@@MBAPBGXZ 1000b54c f i usbh_ehcdmdd_common_topaz_v1:chw.obj
 0001:0000a55c       ?AreTransferParametersValid@CDummyPipe@@MBAHPBUSTRANSFER@@@Z 1000b55c f i usbh_ehcdmdd_common_topaz_v1:chw.obj
 0001:0000a564       ?CheckForDoneTransfers@CDummyPipe@@MAAHXZ 1000b564 f i usbh_ehcdmdd_common_topaz_v1:chw.obj
 0001:0000a56c       ??_GCDummyPipe@@UAAPAXI@Z  1000b56c f i usbh_ehcdmdd_common_topaz_v1:chw.obj
 0001:0000a56c       ??_ECDummyPipe@@UAAPAXI@Z  1000b56c f i usbh_ehcdmdd_common_topaz_v1:chw.obj
 0001:0000a59c       ??0CPeriodicMgr@@QAA@QAVCPhysMem@@K@Z 1000b59c f   usbh_ehcdmdd_common_topaz_v1:chw.obj
 0001:0000a628       ?QueueITD@CPeriodicMgr@@QAAHPAVCITD@@K@Z 1000b628 f   usbh_ehcdmdd_common_topaz_v1:chw.obj
 0001:0000a6c0       ?DeQueueTD@CPeriodicMgr@@QAAHKK@Z 1000b6c0 f   usbh_ehcdmdd_common_topaz_v1:chw.obj
 0001:0000a7c0       ??0CAsyncMgr@@QAA@QAVCPhysMem@@@Z 1000b7c0 f   usbh_ehcdmdd_common_topaz_v1:chw.obj
 0001:0000a808       ?DeInit@CAsyncMgr@@QAAXXZ  1000b808 f   usbh_ehcdmdd_common_topaz_v1:chw.obj
 0001:0000a848       ?SignalCheckForDoneTransfers@CBusyPipeList@@QAAXXZ 1000b848 f   usbh_ehcdmdd_common_topaz_v1:chw.obj
 0001:0000a854       ?CheckForDoneTransfersThread@CBusyPipeList@@AAAKXZ 1000b854 f   usbh_ehcdmdd_common_topaz_v1:chw.obj
 0001:0000a8c4       ?AddToBusyPipeList@CBusyPipeList@@QAAHQAVCPipe@@H@Z 1000b8c4 f   usbh_ehcdmdd_common_topaz_v1:chw.obj
 0001:0000a944       ?RemoveFromBusyPipeList@CBusyPipeList@@QAAXQAVCPipe@@@Z 1000b944 f   usbh_ehcdmdd_common_topaz_v1:chw.obj
 0001:0000a9a8       ?EnableAsyncSchedule@CHW@@QAAHXZ 1000b9a8 f   usbh_ehcdmdd_common_topaz_v1:chw.obj
 0001:0000aa84       ?PowerOnAllPorts@CHW@@QAAHXZ 1000ba84 f   usbh_ehcdmdd_common_topaz_v1:chw.obj
 0001:0000ab30       ?EnterOperationalState@CHW@@QAAXXZ 1000bb30 f   usbh_ehcdmdd_common_topaz_v1:chw.obj
 0001:0000ac20       ?RunStopUSBController@CHW@@QAAXH@Z 1000bc20 f   usbh_ehcdmdd_common_topaz_v1:chw.obj
 0001:0000ad2c       ?StartHostController@CHW@@QAAXXZ 1000bd2c f   usbh_ehcdmdd_common_topaz_v1:chw.obj
 0001:0000ae44       ?StopHostController@CHW@@QAAXXZ 1000be44 f   usbh_ehcdmdd_common_topaz_v1:chw.obj
 0001:0000aefc       ?AsyncBell@CHW@@QAAHXZ     1000befc f   usbh_ehcdmdd_common_topaz_v1:chw.obj
 0001:0000af78       ?PeriodQueueITD@CHW@@QAAHPAVCITD@@K@Z 1000bf78 f   usbh_ehcdmdd_common_topaz_v1:chw.obj
 0001:0000afc4       ?PeriodDeQueueTD@CHW@@QAAHKK@Z 1000bfc4 f   usbh_ehcdmdd_common_topaz_v1:chw.obj
 0001:0000b044       ?CeResumeThread@CHW@@AAAKXZ 1000c044 f   usbh_ehcdmdd_common_topaz_v1:chw.obj
 0001:0000b0dc       ?UpdateFrameCounter@CHW@@AAAXXZ 1000c0dc f   usbh_ehcdmdd_common_topaz_v1:chw.obj
 0001:0000b13c       ?GetFrameNumber@CHW@@UAAHPAK@Z 1000c13c f   usbh_ehcdmdd_common_topaz_v1:chw.obj
 0001:0000b180       ?GetFrameLength@CHW@@UAAHPAG@Z 1000c180 f   usbh_ehcdmdd_common_topaz_v1:chw.obj
 0001:0000b194       ?SetFrameLength@CHW@@UAAHPAXG@Z 1000c194 f   usbh_ehcdmdd_common_topaz_v1:chw.obj
 0001:0000b19c       ?StopAdjustingFrame@CHW@@UAAHXZ 1000c19c f   usbh_ehcdmdd_common_topaz_v1:chw.obj
 0001:0000b1a4       ?DidPortStatusChange@CHW@@UAAHE@Z 1000c1a4 f   usbh_ehcdmdd_common_topaz_v1:chw.obj
 0001:0000b308       ?GetPortStatus@CHW@@UAAHEAAU_USB_HUB_AND_PORT_STATUS@@PAK@Z 1000c308 f   usbh_ehcdmdd_common_topaz_v1:chw.obj
 0001:0000b568       ?RootHubFeature@CHW@@UAAHEEG@Z 1000c568 f   usbh_ehcdmdd_common_topaz_v1:chw.obj
 0001:0000b6cc       ?ResetAndEnablePort@CHW@@UAAHE@Z 1000c6cc f   usbh_ehcdmdd_common_topaz_v1:chw.obj
 0001:0000b91c       ?DisablePort@CHW@@UAAXE@Z  1000c91c f   usbh_ehcdmdd_common_topaz_v1:chw.obj
 0001:0000b9b8       ?WaitForPortStatusChange@CHW@@UAAHPAX@Z 1000c9b8 f   usbh_ehcdmdd_common_topaz_v1:chw.obj
 0001:0000ba24       ?SetCapability@CHW@@UAAKK@Z 1000ca24 f   usbh_ehcdmdd_common_topaz_v1:chw.obj
 0001:0000ba38       ?IsOTGHostDevice@CHW@@UAAHXZ 1000ca38 f   usbh_ehcdmdd_common_topaz_v1:chw.obj
 0001:0000ba6c       ?WakeUpSysIntr@CHW@@UAAXXZ 1000ca6c f   usbh_ehcdmdd_common_topaz_v1:chw.obj
 0001:0000ba74       ?Init@CPeriodicMgr@@QAAHXZ 1000ca74 f   usbh_ehcdmdd_common_topaz_v1:chw.obj
 0001:0000bc5c       ?DeInit@CPeriodicMgr@@QAAXXZ 1000cc5c f   usbh_ehcdmdd_common_topaz_v1:chw.obj
 0001:0000bcd0       ?QueueSITD@CPeriodicMgr@@QAAHPAVCSITD@@K@Z 1000ccd0 f   usbh_ehcdmdd_common_topaz_v1:chw.obj
 0001:0000bd68       ?QueueQHead@CPeriodicMgr@@QAAPAVCQH@@PAV2@EEH@Z 1000cd68 f   usbh_ehcdmdd_common_topaz_v1:chw.obj
 0001:0000bf24       ?DequeueQHead@CPeriodicMgr@@QAAHPAVCQH@@@Z 1000cf24 f   usbh_ehcdmdd_common_topaz_v1:chw.obj
 0001:0000c034       ?Init@CAsyncMgr@@QAAHXZ    1000d034 f   usbh_ehcdmdd_common_topaz_v1:chw.obj
 0001:0000c0c4       ?QueueQH@CAsyncMgr@@QAAPAVCQH@@PAV2@@Z 1000d0c4 f   usbh_ehcdmdd_common_topaz_v1:chw.obj
 0001:0000c174       ?DequeueQHead@CAsyncMgr@@QAAHPAVCQH@@@Z 1000d174 f   usbh_ehcdmdd_common_topaz_v1:chw.obj
 0001:0000c274       ?DeInit@CBusyPipeList@@QAAXXZ 1000d274 f   usbh_ehcdmdd_common_topaz_v1:chw.obj
 0001:0000c2e8       ?CheckForDoneTransfersThreadStub@CBusyPipeList@@CAKPAX@Z 1000d2e8 f   usbh_ehcdmdd_common_topaz_v1:chw.obj
 0001:0000c2ec       ?ConfigureHS@CHW@@QAAHXZ   1000d2ec f   usbh_ehcdmdd_common_topaz_v1:chw.obj
 0001:0000c594       ?DeInitialize@CHW@@UAAXXZ  1000d594 f   usbh_ehcdmdd_common_topaz_v1:chw.obj
 0001:0000c6b0       ?AsyncDequeueQH@CHW@@QAAHPAVCQH@@@Z 1000d6b0 f   usbh_ehcdmdd_common_topaz_v1:chw.obj
 0001:0000c6d4       ?PeriodQueueSITD@CHW@@QAAHPAVCSITD@@K@Z 1000d6d4 f   usbh_ehcdmdd_common_topaz_v1:chw.obj
 0001:0000c720       ?CeResumeThreadStub@CHW@@CAKPAX@Z 1000d720 f   usbh_ehcdmdd_common_topaz_v1:chw.obj
 0001:0000c724       ?EnterLowPowerMode@CHW@@QAAXXZ 1000d724 f   usbh_ehcdmdd_common_topaz_v1:chw.obj
 0001:0000c8fc       ?PowerMgmtCallback@CHW@@UAAXH@Z 1000d8fc f   usbh_ehcdmdd_common_topaz_v1:chw.obj
 0001:0000cbe4       ??1CPeriodicMgr@@QAA@XZ    1000dbe4 f   usbh_ehcdmdd_common_topaz_v1:chw.obj
 0001:0000cc14       ?Init@CBusyPipeList@@QAAHXZ 1000dc14 f   usbh_ehcdmdd_common_topaz_v1:chw.obj
 0001:0000cca0       ??0CHW@@QAA@SAEKKQAVCPhysMem@@PAXPBG@Z 1000dca0 f   usbh_ehcdmdd_common_topaz_v1:chw.obj
 0001:0000cdfc       ??1CHW@@UAA@XZ             1000ddfc f   usbh_ehcdmdd_common_topaz_v1:chw.obj
 0001:0000cec4       ?UsbInterruptThread@CHW@@AAAKXZ 1000dec4 f   usbh_ehcdmdd_common_topaz_v1:chw.obj
 0001:0000d83c       ??_ECHW@@UAAPAXI@Z         1000e83c f i usbh_ehcdmdd_common_topaz_v1:chw.obj
 0001:0000d83c       ??_GCHW@@UAAPAXI@Z         1000e83c f i usbh_ehcdmdd_common_topaz_v1:chw.obj
 0001:0000d860       ?UsbInterruptThreadStub@CHW@@CAKPAX@Z 1000e860 f   usbh_ehcdmdd_common_topaz_v1:chw.obj
 0001:0000d878       ?Initialize@CHW@@UAAHXZ    1000e878 f   usbh_ehcdmdd_common_topaz_v1:chw.obj
 0001:0000d9dc       ??0CTransfer@@QAA@QAVCPipe@@QAVCPhysMem@@PAUSTRANSFER@@@Z 1000e9dc f   usbh_ehcdmdd_common_topaz_v1:trans.obj
 0001:0000da48       ??1CTransfer@@UAA@XZ       1000ea48 f   usbh_ehcdmdd_common_topaz_v1:trans.obj
 0001:0000da98       ?Init@CTransfer@@UAAHXZ    1000ea98 f   usbh_ehcdmdd_common_topaz_v1:trans.obj
 0001:0000dc04       ??0CIsochTransfer@@QAA@QAVCIsochronousPipe@@QAVCEhcd@@PAUSTRANSFER@@@Z 1000ec04 f   usbh_ehcdmdd_common_topaz_v1:trans.obj
 0001:0000dc58       ?ArmTD@CITransfer@@QAAHXZ  1000ec58 f   usbh_ehcdmdd_common_topaz_v1:trans.obj
 0001:0000de48       ?AddTransfer@CITransfer@@UAAHXZ 1000ee48 f   usbh_ehcdmdd_common_topaz_v1:trans.obj
 0001:0000df04       ?ScheduleTD@CITransfer@@UAAHKK@Z 1000ef04 f   usbh_ehcdmdd_common_topaz_v1:trans.obj
 0001:0000dfcc       ?IsTransferDone@CITransfer@@UAAHKK@Z 1000efcc f   usbh_ehcdmdd_common_topaz_v1:trans.obj
 0001:0000e22c       ?AbortTransfer@CITransfer@@UAAHXZ 1000f22c f   usbh_ehcdmdd_common_topaz_v1:trans.obj
 0001:0000e394       ?DoneTransfer@CITransfer@@UAAHKK@Z 1000f394 f   usbh_ehcdmdd_common_topaz_v1:trans.obj
 0001:0000e4a0       ?DoneTransfer@CSITransfer@@UAAHKK@Z 1000f4a0 f   usbh_ehcdmdd_common_topaz_v1:trans.obj
 0001:0000e5ac       ??_GCIsochTransfer@@UAAPAXI@Z 1000f5ac f i usbh_ehcdmdd_common_topaz_v1:trans.obj
 0001:0000e5ac       ??_ECIsochTransfer@@UAAPAXI@Z 1000f5ac f i usbh_ehcdmdd_common_topaz_v1:trans.obj
 0001:0000e5dc       ??_GCTransfer@@UAAPAXI@Z   1000f5dc f i usbh_ehcdmdd_common_topaz_v1:trans.obj
 0001:0000e5dc       ??_ECTransfer@@UAAPAXI@Z   1000f5dc f i usbh_ehcdmdd_common_topaz_v1:trans.obj
 0001:0000e600       ?AddTransfer@CQTransfer@@UAAHXZ 1000f600 f   usbh_ehcdmdd_common_topaz_v1:trans.obj
 0001:0000ea48       ?AbortTransfer@CQTransfer@@QAAHXZ 1000fa48 f   usbh_ehcdmdd_common_topaz_v1:trans.obj
 0001:0000ea8c       ?IsTransferDone@CQTransfer@@QAAHXZ 1000fa8c f   usbh_ehcdmdd_common_topaz_v1:trans.obj
 0001:0000eaec       ??0CITransfer@@QAA@QAVCIsochronousPipe@@QAVCEhcd@@PAUSTRANSFER@@@Z 1000faec f   usbh_ehcdmdd_common_topaz_v1:trans.obj
 0001:0000eb14       ??1CITransfer@@UAA@XZ      1000fb14 f   usbh_ehcdmdd_common_topaz_v1:trans.obj
 0001:0000ebb0       ??0CSITransfer@@QAA@QAVCIsochronousPipe@@QAVCEhcd@@PAUSTRANSFER@@@Z 1000fbb0 f   usbh_ehcdmdd_common_topaz_v1:trans.obj
 0001:0000ebd8       ?ArmTD@CSITransfer@@QAAHXZ 1000fbd8 f   usbh_ehcdmdd_common_topaz_v1:trans.obj
 0001:0000ece4       ?AddTransfer@CSITransfer@@UAAHXZ 1000fce4 f   usbh_ehcdmdd_common_topaz_v1:trans.obj
 0001:0000ed88       ?ScheduleTD@CSITransfer@@UAAHKK@Z 1000fd88 f   usbh_ehcdmdd_common_topaz_v1:trans.obj
 0001:0000ee50       ?IsTransferDone@CSITransfer@@UAAHKK@Z 1000fe50 f   usbh_ehcdmdd_common_topaz_v1:trans.obj
 0001:0000f0a8       ?AbortTransfer@CSITransfer@@UAAHXZ 100100a8 f   usbh_ehcdmdd_common_topaz_v1:trans.obj
 0001:0000f1f0       ??1CQTransfer@@UAA@XZ      100101f0 f   usbh_ehcdmdd_common_topaz_v1:trans.obj
 0001:0000f24c       ?DoneTransfer@CQTransfer@@QAAHXZ 1001024c f   usbh_ehcdmdd_common_topaz_v1:trans.obj
 0001:0000f3e0       ??_ECITransfer@@UAAPAXI@Z  100103e0 f i usbh_ehcdmdd_common_topaz_v1:trans.obj
 0001:0000f3e0       ??_GCITransfer@@UAAPAXI@Z  100103e0 f i usbh_ehcdmdd_common_topaz_v1:trans.obj
 0001:0000f404       ??1CSITransfer@@UAA@XZ     10010404 f   usbh_ehcdmdd_common_topaz_v1:trans.obj
 0001:0000f4a0       ??_ECSITransfer@@UAAPAXI@Z 100104a0 f i usbh_ehcdmdd_common_topaz_v1:trans.obj
 0001:0000f4a0       ??_GCSITransfer@@UAAPAXI@Z 100104a0 f i usbh_ehcdmdd_common_topaz_v1:trans.obj
 0001:0000f4c4       ??2CNextLinkPointer@@SAPAXIQAVCPhysMem@@@Z 100104c4 f   usbh_ehcdmdd_common_topaz_v1:ctd.obj
 0001:0000f560       ??3CNextLinkPointer@@SAXPAX@Z 10010560 f   usbh_ehcdmdd_common_topaz_v1:ctd.obj
 0001:0000f564       ??0CITD@@QAA@PAVCITransfer@@@Z 10010564 f   usbh_ehcdmdd_common_topaz_v1:ctd.obj
 0001:0000f5e8       ?ReInit@CITD@@QAAXPAVCITransfer@@@Z 100105e8 f   usbh_ehcdmdd_common_topaz_v1:ctd.obj
 0001:0000f660       ?SetIOC@CITD@@QAAXH@Z      10010660 f   usbh_ehcdmdd_common_topaz_v1:ctd.obj
 0001:0000f6e0       ?IssueTransfer@CITD@@QAAKKPAK0HH@Z 100106e0 f   usbh_ehcdmdd_common_topaz_v1:ctd.obj
 0001:0000f96c       ??0CSITD@@QAA@PAVCSITransfer@@PAV0@@Z 1001096c f   usbh_ehcdmdd_common_topaz_v1:ctd.obj
 0001:0000fa3c       ?ReInit@CSITD@@QAAXPAVCSITransfer@@PAV1@@Z 10010a3c f   usbh_ehcdmdd_common_topaz_v1:ctd.obj
 0001:0000fb00       ??0CQTD@@QAA@PAVCQTransfer@@PAVCQH@@@Z 10010b00 f   usbh_ehcdmdd_common_topaz_v1:ctd.obj
 0001:0000fb90       ?IssueTransfer@CQTD@@QAAKKHKPAUPhysBufferArray@@H@Z 10010b90 f   usbh_ehcdmdd_common_topaz_v1:ctd.obj
 0001:0000fd38       ??0CQH@@QAA@PAVCPipe@@@Z   10010d38 f   usbh_ehcdmdd_common_topaz_v1:ctd.obj
 0001:0000ff2c       ?IssueTransfer@CSITD@@QAAKKKKHH@Z 10010f2c f   usbh_ehcdmdd_common_topaz_v1:ctd.obj
 0001:00010160       ?QueueNextTD@CQTD@@QAAPAV1@PAV1@@Z 10011160 f   usbh_ehcdmdd_common_topaz_v1:ctd.obj
 0001:00010184       ?QueueTD@CQH@@QAAHPAVCQTD@@@Z 10011184 f   usbh_ehcdmdd_common_topaz_v1:ctd.obj
 0001:000101d8       HcdPdd_DllMain             100111d8 f   usbh_ehcdpdd_common_topaz_v1:system.obj
 0001:000101e0       ConfigureEHCICard          100111e0 f   usbh_ehcdpdd_common_topaz_v1:system.obj
 0001:00010654       HcdPdd_Init                10011654 f   usbh_ehcdpdd_common_topaz_v1:system.obj
 0001:000106d8       HcdPdd_CheckConfigPower    100116d8 f   usbh_ehcdpdd_common_topaz_v1:system.obj
 0001:000106dc       HcdPdd_PowerUp             100116dc f   usbh_ehcdpdd_common_topaz_v1:system.obj
 0001:000106e4       HcdPdd_PowerDown           100116e4 f   usbh_ehcdpdd_common_topaz_v1:system.obj
 0001:000106ec       HcdPdd_Deinit              100116ec f   usbh_ehcdpdd_common_topaz_v1:system.obj
 0001:0001077c       HcdPdd_Open                1001177c f   usbh_ehcdpdd_common_topaz_v1:system.obj
 0001:00010780       HcdPdd_Close               10011780 f   usbh_ehcdpdd_common_topaz_v1:system.obj
 0001:00010788       HcdPdd_Read                10011788 f   usbh_ehcdpdd_common_topaz_v1:system.obj
 0001:00010790       HcdPdd_Write               10011790 f   usbh_ehcdpdd_common_topaz_v1:system.obj
 0001:00010798       HcdPdd_Seek                10011798 f   usbh_ehcdpdd_common_topaz_v1:system.obj
 0001:000107a0       HcdPdd_IOControl           100117a0 f   usbh_ehcdpdd_common_topaz_v1:system.obj
 0001:000107dc       HcdPdd_InitiatePowerUp     100117dc f   usbh_ehcdpdd_common_topaz_v1:system.obj
 0001:000107e0       KernelIoControl            100117e0 f   coredll:COREDLL.dll
 0001:000107f0       Sleep                      100117f0 f   coredll:COREDLL.dll
 0001:00010800       StringCchCopyW             10011800 f   coredll:COREDLL.dll
 0001:00010810       InterlockedCompareExchange 10011810 f   coredll:COREDLL.dll
 0001:00010820       GetLastError               10011820 f   coredll:COREDLL.dll
 0001:00010830       MapViewOfFile              10011830 f   coredll:COREDLL.dll
 0001:00010840       CreateFileMappingW         10011840 f   coredll:COREDLL.dll
 0001:00010850       CloseHandle                10011850 f   coredll:COREDLL.dll
 0001:00010860       DeleteCriticalSection      10011860 f   coredll:COREDLL.dll
 0001:00010870       InitializeCriticalSection  10011870 f   coredll:COREDLL.dll
 0001:00010880       DisableThreadLibraryCalls  10011880 f   coredll:COREDLL.dll
 0001:00010890       RegCloseKey                10011890 f   coredll:COREDLL.dll
 0001:000108a0       RegQueryValueExW           100118a0 f   coredll:COREDLL.dll
 0001:000108b0       OpenDeviceKey              100118b0 f   coredll:COREDLL.dll
 0001:000108c0       LeaveCriticalSection       100118c0 f   coredll:COREDLL.dll
 0001:000108d0       EnterCriticalSection       100118d0 f   coredll:COREDLL.dll
 0001:000108e0       RegOpenKeyExW              100118e0 f   coredll:COREDLL.dll
 0001:000108f0       EventModify                100118f0 f   coredll:COREDLL.dll
 0001:00010900       LocalAlloc                 10011900 f   coredll:COREDLL.dll
 0001:00010910       LocalFree                  10011910 f   coredll:COREDLL.dll
 0001:00010920       WaitForSingleObject        10011920 f   coredll:COREDLL.dll
 0001:00010930       FreePhysMem                10011930 f   coredll:COREDLL.dll
 0001:00010940       CreateEventW               10011940 f   coredll:COREDLL.dll
 0001:00010950       AllocPhysMem               10011950 f   coredll:COREDLL.dll
 0001:00010960       SetLastError               10011960 f   coredll:COREDLL.dll
 0001:00010970       FreeLibrary                10011970 f   coredll:COREDLL.dll
 0001:00010980       GetProcAddressW            10011980 f   coredll:COREDLL.dll
 0001:00010990       LoadLibraryW               10011990 f   coredll:COREDLL.dll
 0001:000109a0       LoadDriver                 100119a0 f   coredll:COREDLL.dll
 0001:000109b0       StringCchCatW              100119b0 f   coredll:COREDLL.dll
 0001:000109c0       CeGetThreadPriority        100119c0 f   coredll:COREDLL.dll
 0001:000109d0       CeSetThreadPriority        100119d0 f   coredll:COREDLL.dll
 0001:000109e0       CreateThread               100119e0 f   coredll:COREDLL.dll
 0001:000109f0       __GetUserKData             100119f0 f   coredll:COREDLL.dll
 0001:00010a00       GetTickCount               10011a00 f   coredll:COREDLL.dll
 0001:00010a10       RaiseException             10011a10 f   coredll:COREDLL.dll
 0001:00010a20       WaitForMultipleObjects     10011a20 f   coredll:COREDLL.dll
 0001:00010a30       SetInterruptEvent          10011a30 f   coredll:COREDLL.dll
 0001:00010a40       TerminateThread            10011a40 f   coredll:COREDLL.dll
 0001:00010a50       InterruptDisable           10011a50 f   coredll:COREDLL.dll
 0001:00010a60       InterruptInitialize        10011a60 f   coredll:COREDLL.dll
 0001:00010a70       InterruptDone              10011a70 f   coredll:COREDLL.dll
 0001:00010a80       ExitThread                 10011a80 f   coredll:COREDLL.dll
 0001:00010a90       FreeIntChainHandler        10011a90 f   coredll:COREDLL.dll
 0001:00010aa0       StringCchCopyNW            10011aa0 f   coredll:COREDLL.dll
 0001:00010ab0       DDKReg_GetIsrInfo          10011ab0 f   coredll:COREDLL.dll
 0001:00010ac0       DDKReg_GetWindowInfo       10011ac0 f   coredll:COREDLL.dll
 0001:00010ad0       StallExecution             10011ad0 f   ceddk:CEDDK.dll
 0001:00010ae0       BusTransBusAddrToVirtual   10011ae0 f   ceddk:CEDDK.dll
 0001:00010af0       HalFreeCommonBuffer        10011af0 f   ceddk:CEDDK.dll
 0001:00010b00       HalAllocateCommonBuffer    10011b00 f   ceddk:CEDDK.dll
 0001:00010b10       CloseBusAccessHandle       10011b10 f   ceddk:CEDDK.dll
 0001:00010b20       CreateBusAccessHandle      10011b20 f   ceddk:CEDDK.dll
 0001:00010b30       DDKIomuxSelectInput        10011b30 f   cspddk:CSPDDK.dll
 0001:00010b40       DDKGpioWriteDataPin        10011b40 f   cspddk:CSPDDK.dll
 0001:00010b50       DDKGpioSetConfig           10011b50 f   cspddk:CSPDDK.dll
 0001:00010b60       DDKIomuxSetPadConfig       10011b60 f   cspddk:CSPDDK.dll
 0001:00010b70       DDKIomuxSetPinMux          10011b70 f   cspddk:CSPDDK.dll
 0001:00010b80       DDKClockSetGatingMode      10011b80 f   cspddk:CSPDDK.dll
 0001:00010b90       DDKClockGetGatingMode      10011b90 f   cspddk:CSPDDK.dll
 0001:00010ba0       DDKClockConfigBaud         10011ba0 f   cspddk:CSPDDK.dll
 0001:00010ca8       _DllMainCRTStartup         10011ca8 f   corelib0:pegdmain.obj
 0001:00010cd4       __GSHandlerCheckCommon     10011cd4 f   corelib0:gshandler.obj
 0001:00010d0c       __GSHandlerCheck           10011d0c f   corelib0:gshandler.obj
 0001:00010d2c       __security_init_cookie     10011d2c f   corelib0:seccinit.obj
 0001:00010d78       __security_check_cookie    10011d78 f   corelib0:armsecgs.obj
 0001:00010d88       __gsfailure                10011d88     corelib0:armsecgs.obj
 0001:00010e8c       _cexit                     10011e8c f   corelib0:cexit.obj
 0001:00010e9c       _initterm                  10011e9c f   corelib0:crt0dat.obj
 0001:00010ec8       _cinit                     10011ec8 f   corelib0:crt0dat.obj
 0001:00010f28       __crt_ExitProcess          10011f28 f   corelib0:exitproc_proxy.obj
 0001:00010f34       ??3@YAXPAX@Z               10011f34 f   corelib1:COREDLL.dll
 0001:00010f44       ??2@YAPAXI@Z               10011f44 f   corelib1:COREDLL.dll
 0001:00010f54       _purecall                  10011f54 f   corelib1:COREDLL.dll
 0001:00010f64       memset                     10011f64 f   corelib1:COREDLL.dll
 0001:00010f74       memcpy                     10011f74 f   corelib1:COREDLL.dll
 0001:00010f84       wcslen                     10011f84 f   corelib1:COREDLL.dll
 0001:00010f94       memcmp                     10011f94 f   corelib1:COREDLL.dll
 0001:00010fa4       __C_specific_handler       10011fa4 f   corelib1:COREDLL.dll
 0001:00010fb4       __rt_sdiv                  10011fb4 f   corelib1:COREDLL.dll
 0001:00010fc4       __rt_udiv                  10011fc4 f   corelib1:COREDLL.dll
 0001:00010fd4       free                       10011fd4 f   corelib1:COREDLL.dll
 0001:00010fe4       malloc                     10011fe4 f   corelib1:COREDLL.dll
 0001:00010ff4       _XcptFilter                10011ff4 f   corelib1:COREDLL.dll
 0001:00011004       __security_gen_cookie2     10012004 f   corelib1:COREDLL.dll
 0001:00011014       __report_gsfailure         10012014 f   corelib1:COREDLL.dll
 0001:00011024       TerminateProcess           10012024 f   coredll:COREDLL.dll
 0001:000111b8       __IMPORT_DESCRIPTOR_COREDLL 100121b8     coredll:COREDLL.dll
 0001:000111cc       __IMPORT_DESCRIPTOR_CEDDK  100121cc     ceddk:CEDDK.dll
 0001:000111e0       __IMPORT_DESCRIPTOR_CSPDDK 100121e0     cspddk:CSPDDK.dll
 0001:000111f4       __NULL_IMPORT_DESCRIPTOR   100121f4     coredll:COREDLL.dll
 0002:00000000       __imp_CloseBusAccessHandle 10013000     ceddk:CEDDK.dll
 0002:00000004       __imp_HalAllocateCommonBuffer 10013004     ceddk:CEDDK.dll
 0002:00000008       __imp_HalFreeCommonBuffer  10013008     ceddk:CEDDK.dll
 0002:0000000c       __imp_BusTransBusAddrToVirtual 1001300c     ceddk:CEDDK.dll
 0002:00000010       __imp_StallExecution       10013010     ceddk:CEDDK.dll
 0002:00000014       __imp_CreateBusAccessHandle 10013014     ceddk:CEDDK.dll
 0002:00000018       \177CEDDK_NULL_THUNK_DATA  10013018     ceddk:CEDDK.dll
 0002:0000001c       __imp_CloseHandle          1001301c     coredll:COREDLL.dll
 0002:00000020       __imp_DeleteCriticalSection 10013020     coredll:COREDLL.dll
 0002:00000024       __imp_InitializeCriticalSection 10013024     coredll:COREDLL.dll
 0002:00000028       __imp_DisableThreadLibraryCalls 10013028     coredll:COREDLL.dll
 0002:0000002c       __imp_RegCloseKey          1001302c     coredll:COREDLL.dll
 0002:00000030       __imp_RegQueryValueExW     10013030     coredll:COREDLL.dll
 0002:00000034       __imp_OpenDeviceKey        10013034     coredll:COREDLL.dll
 0002:00000038       __imp_LeaveCriticalSection 10013038     coredll:COREDLL.dll
 0002:0000003c       __imp_EnterCriticalSection 1001303c     coredll:COREDLL.dll
 0002:00000040       __imp_RegOpenKeyExW        10013040     coredll:COREDLL.dll
 0002:00000044       __imp_EventModify          10013044     coredll:COREDLL.dll
 0002:00000048       __imp_LocalAlloc           10013048     coredll:COREDLL.dll
 0002:0000004c       __imp_LocalFree            1001304c     coredll:COREDLL.dll
 0002:00000050       __imp_WaitForSingleObject  10013050     coredll:COREDLL.dll
 0002:00000054       __imp_FreePhysMem          10013054     coredll:COREDLL.dll
 0002:00000058       __imp_CreateEventW         10013058     coredll:COREDLL.dll
 0002:0000005c       __imp_AllocPhysMem         1001305c     coredll:COREDLL.dll
 0002:00000060       __imp_SetLastError         10013060     coredll:COREDLL.dll
 0002:00000064       __imp_FreeLibrary          10013064     coredll:COREDLL.dll
 0002:00000068       __imp_CreateFileMappingW   10013068     coredll:COREDLL.dll
 0002:0000006c       __imp_LoadLibraryW         1001306c     coredll:COREDLL.dll
 0002:00000070       __imp_LoadDriver           10013070     coredll:COREDLL.dll
 0002:00000074       __imp_StringCchCatW        10013074     coredll:COREDLL.dll
 0002:00000078       __imp_CeGetThreadPriority  10013078     coredll:COREDLL.dll
 0002:0000007c       __imp_CeSetThreadPriority  1001307c     coredll:COREDLL.dll
 0002:00000080       __imp_CreateThread         10013080     coredll:COREDLL.dll
 0002:00000084       __imp___GetUserKData       10013084     coredll:COREDLL.dll
 0002:00000088       __imp_GetTickCount         10013088     coredll:COREDLL.dll
 0002:0000008c       __imp_RaiseException       1001308c     coredll:COREDLL.dll
 0002:00000090       __imp_WaitForMultipleObjects 10013090     coredll:COREDLL.dll
 0002:00000094       __imp_SetInterruptEvent    10013094     coredll:COREDLL.dll
 0002:00000098       __imp_TerminateThread      10013098     coredll:COREDLL.dll
 0002:0000009c       __imp_InterruptDisable     1001309c     coredll:COREDLL.dll
 0002:000000a0       __imp_InterruptInitialize  100130a0     coredll:COREDLL.dll
 0002:000000a4       __imp_InterruptDone        100130a4     coredll:COREDLL.dll
 0002:000000a8       __imp_ExitThread           100130a8     coredll:COREDLL.dll
 0002:000000ac       __imp_FreeIntChainHandler  100130ac     coredll:COREDLL.dll
 0002:000000b0       __imp_StringCchCopyNW      100130b0     coredll:COREDLL.dll
 0002:000000b4       __imp_DDKReg_GetIsrInfo    100130b4     coredll:COREDLL.dll
 0002:000000b8       __imp_DDKReg_GetWindowInfo 100130b8     coredll:COREDLL.dll
 0002:000000bc       __imp_MapViewOfFile        100130bc     coredll:COREDLL.dll
 0002:000000c0       __imp_GetLastError         100130c0     coredll:COREDLL.dll
 0002:000000c4       __imp_InterlockedCompareExchange 100130c4     coredll:COREDLL.dll
 0002:000000c8       __imp_StringCchCopyW       100130c8     coredll:COREDLL.dll
 0002:000000cc       __imp_Sleep                100130cc     coredll:COREDLL.dll
 0002:000000d0       __imp_GetProcAddressW      100130d0     coredll:COREDLL.dll
 0002:000000d4       __imp_KernelIoControl      100130d4     coredll:COREDLL.dll
 0002:000000d8       __imp___report_gsfailure   100130d8     corelib1:COREDLL.dll
 0002:000000dc       __imp___security_gen_cookie2 100130dc     corelib1:COREDLL.dll
 0002:000000e0       __imp__XcptFilter          100130e0     corelib1:COREDLL.dll
 0002:000000e4       __imp_malloc               100130e4     corelib1:COREDLL.dll
 0002:000000e8       __imp_free                 100130e8     corelib1:COREDLL.dll
 0002:000000ec       __imp___rt_udiv            100130ec     corelib1:COREDLL.dll
 0002:000000f0       __imp___rt_sdiv            100130f0     corelib1:COREDLL.dll
 0002:000000f4       __imp_??3@YAXPAX@Z         100130f4     corelib1:COREDLL.dll
 0002:000000f8       __imp_??2@YAPAXI@Z         100130f8     corelib1:COREDLL.dll
 0002:000000fc       __imp__purecall            100130fc     corelib1:COREDLL.dll
 0002:00000100       __imp_memset               10013100     corelib1:COREDLL.dll
 0002:00000104       __imp_memcpy               10013104     corelib1:COREDLL.dll
 0002:00000108       __imp_wcslen               10013108     corelib1:COREDLL.dll
 0002:0000010c       __imp_memcmp               1001310c     corelib1:COREDLL.dll
 0002:00000110       __imp___C_specific_handler 10013110     corelib1:COREDLL.dll
 0002:00000114       __imp_TerminateProcess     10013114     coredll:COREDLL.dll
 0002:00000118       \177COREDLL_NULL_THUNK_DATA 10013118     coredll:COREDLL.dll
 0002:0000011c       __imp_DDKClockConfigBaud   1001311c     cspddk:CSPDDK.dll
 0002:00000120       __imp_DDKClockGetGatingMode 10013120     cspddk:CSPDDK.dll
 0002:00000124       __imp_DDKClockSetGatingMode 10013124     cspddk:CSPDDK.dll
 0002:00000128       __imp_DDKIomuxSetPinMux    10013128     cspddk:CSPDDK.dll
 0002:0000012c       __imp_DDKIomuxSetPadConfig 1001312c     cspddk:CSPDDK.dll
 0002:00000130       __imp_DDKGpioSetConfig     10013130     cspddk:CSPDDK.dll
 0002:00000134       __imp_DDKGpioWriteDataPin  10013134     cspddk:CSPDDK.dll
 0002:00000138       __imp_DDKIomuxSelectInput  10013138     cspddk:CSPDDK.dll
 0002:0000013c       \177CSPDDK_NULL_THUNK_DATA 1001313c     cspddk:CSPDDK.dll
 0002:00000140       ?gc_HcdFuncs@@3U_HCD_FUNCS@@A 10013140     usbh_usb2com_common_topaz_v1:hcddrv.obj
 0002:00000178       ?cszPipeType@?1??GetPipeType@CInterruptPipe@@UBAPBGXZ@4PBGB 10013178     usbh_ehcdmdd_common_topaz_v1:cpipe.obj
 0002:0000017c       ?cszPipeType@?1??GetPipeType@CIsochronousPipe@@UBAPBGXZ@4PBGB 1001317c     usbh_ehcdmdd_common_topaz_v1:cpipe.obj
 0002:00000180       ?CMASKS@USB2lib@@0PAEA     10013180     usbh_ehcdmdd_common_topaz_v1:usb2lib.obj
 0002:00000188       ?periodTable@CPeriodicMgr@@0PAU_PERIOD_TABLE@@A 10013188     usbh_ehcdmdd_common_topaz_v1:chw.obj
 0002:00000248       ?cszPipeType@?1??GetPipeType@CDummyPipe@@MBAPBGXZ@4PBGB 10013248     usbh_ehcdmdd_common_topaz_v1:chw.obj
 0002:0000024c       __security_cookie          1001324c     corelib0:seccinit.obj
 0002:00000250       __security_cookie_complement 10013250     corelib0:seccinit.obj
 0002:00000260       m_hUSBClockGatingHandle    10013260     i_usbclock.obj
 0002:00000264       pUSBClkGating              10013264     i_usbclock.obj
 0002:00000268       g_IstThreadPriority        10013268     usbh_usb2com_common_topaz_v1:hcddrv.obj
 0002:0000026c       ?g_CSection@@3UCRITICAL_SECTION@@A 1001326c     usbh_usb2com_common_topaz_v1:hcddrv.obj
 0002:00000280       g_dwContext                10013280     usbh_usb2com_common_topaz_v1:hcddrv.obj
 0002:00000284       ?ghDetach@@3PAXA           10013284     usbh_usb2com_common_topaz_v1:cdevice.obj
 0002:00000288       ?m_dwGlobalTransferID@CTransfer@@1KA 10013288     usbh_ehcdmdd_common_topaz_v1:trans.obj
 0002:0000028c       _exitflag                  1001328c     corelib0:cexit.obj
 0002:0000028e       gSel                       1001328e     <common>
 0002:000002a0       gszOTGGroup                100132a0     <common>
 0002:000002dc       gRegs                      100132dc     <common>
 0002:000002e0       gdwOTGSupport              100132e0     <common>
 0002:000002e4       __onexitend                100132e4     <common>
 0002:000002e8       __onexitbegin              100132e8     <common>
 0002:000002ec       _pRawDllMain               100132ec     <common>

 entry point at        0001:00010ca8

 Static symbols

 0001:00000930       InitializeHost2Mux         10001930 f   i_hwinit.obj
 0001:000009e4       ConfigH2                   100019e4 f   i_hwinit.obj
 0001:00001344       HcdDisableDevice           10002344 f   usbh_usb2com_common_topaz_v1:hcddrv.obj
 0001:00001358       HcdSuspendResume           10002358 f   usbh_usb2com_common_topaz_v1:hcddrv.obj
 0001:00010244       InitializeEHCI             10011244 f   usbh_ehcdpdd_common_topaz_v1:system.obj
 0001:00010bb8       _DllMainCRTStartupHelper   10011bb8 f   corelib0:pegdmain.obj
 0001:00010dcc       doexit                     10011dcc f   corelib0:cexit.obj
